:090000000217DB0248B32573006E
:10000B000249E9E4FFFE120731600C0FEF70010E9D
:0F001B0009E970F20A80EF220249F85322E0222D
:07002B00024FF943EA4022F5
:100033000241559000E27406F09000E07400F090E5
:1000430000E27412F07581AA1238020217DB75A858
:10005300009000E27406F09000E07480F09000E2FB
:10006300740CF00217DB244750524D430000020486
:1000730037E86480F8E933E83360110460F0ED3366
:10008300EC337009E8FCE9FDEAFEEBFF220460DED5
:10009300D3EB9FEA9EE99DE8C2E78CF0C2F795F0A7
:1000A300400CE8CCF8E9CDF9EACEFAEBCFFB120429
:1000B3000285D0F05804700320D5B3E804700750CC
:1000C30002B2D502044192D5EC0460F7E4CCC0E05F
:1000D300C398F8603B94186008400DD0E0FB02041D
:1000E30019E4FBFAC9FC8028E830E406E4C9FBE420
:1000F300CAFCE830E305E4C9CACBFCE85407601046
:10010300F8C3E913F9EA13FAEB13FBEC13FCD8F188
:1001130030F52FC3E49CFCEF9BFFEE9AFEED99FDB7
:10012300D0E0FBEF4E4D4C701222DB0302043EEC99
:100133002CFCEF33FFEE33FEED33FDED30E7EB0246
:100143000419EF2BFFEE3AFEED39FDD0E0FB50131F
:100153000BBB0003020441ED13FDEE13FEEF13FF8F
:10016300EC13FC020419EC4D6011E8497017ED33F0
:10017300EC3304600DE4FCFFFEFD22E933E83304B5
:1001830070F802043712040258046009E4CC248195
:10019300500628500902044128400302043EC0E0EF
:1001A300EB4A7044B98006D0E0FB02042DEF4E7099
:1001B3001CBD8008EBFFEAFEE9FD80EBE98DF0A4AE
:1001C300FEE5F0020252E9CDF9EAFEEBFFEF89F01A
:1001D300A4FCE5F0CE89F0A42EFFE435F0CD89F040
:1001E300A42DFEE435F08067EF4E7005BD80D78007
:1001F300C3EF8BF0A4ACF0EE8BF0A42CFCE435F051
:10020300F8EF8AF0A42CE5F038FCE433CB8DF0A4AE
:100213002CFCE5F03BF8EE8AF0A42CFCE5F038F872
:10022300E433CF89F0A42CFCE5F038CF3400CE8939
:10023300F0A42FFFE5F03EFEE433C98DF0A42EFEBB
:10024300E5F039CD8AF0A42FFFE5F03EFEE43DFD55
:1002530033D0E0FB50070BBB000F020441EC2CFC36
:10026300EF33FFEE33FEED33FD020419020441ECDC
:100273005D046005E8590470030204371204025850
:100283000460F6EC4860F2EC7004FDFEFF22C860E7
:10029300DB2481C85009C3986002500602043E98CB
:1002A30050CAF582E9294B4A7005AB8202042D75C9
:1002B300F0007C1A7880C3EF9BEE9AED99400DC352
:1002C300EF9BFFEE9AFEED99FDE842F0DC23ACF0E4
:1002D300D0E0FFD0E0FED0E0FDAB8220E7101BEBC7
:1002E30060BAEC2CFCEF33FFEE33FEED33FD02047A
:1002F30019E803F830E705C0F075F000EF2FFFEEC3
:1003030033FEED33FD40B830E7C280AA74F8CC6405
:1003130080CCC86480C8F582046043C3EB9FF5F0CA
:10032300EA9E42F0E99D42F0E89C45F060305018A7
:10033300E5825FFFE582F42B5582FB50210ABA0068
:100343001D09B90019088016E5825BFBE582F42FCD
:100353005582FF50090EBE00050DBD00010CC3EB15
:100363009FF5F0EA9E42F0E99D42F0E89C45F0607B
:1003730007CC4820E701B3EC22ED33EC33600A04E9
:100383007003BD8004ECB2E7FC2275F020800E758B
:10039300F010800575F0087D007E007F003392D554
:1003A30030D503120959EC334010EF33FFEE33FE1F
:1003B300ED33FDEC33FCD5F0ED22E5F0247EA2D540
:1003C30013CC92E7CDCEFF22EDD2E7CD33EC3392BF
:1003D300D524814006E4FFFEFDFC22FCE4CFCECD14
:1003E300CC24E0501174FF80EDC3CC13CCCD13CDDE
:1003F300CE13CECF13CF0470F030D5DE020959E906
:10040300D2E7C933E833F892D5EDD2E7CD33EC33F5
:10041300FC5002B2D522EC30E7100FBF000C0EBE29
:1004230000080DBD00040BEB6014A2D5EB13FCED2B
:1004330092E7FD2274FFFCFDFEFF22E480F8A2D5C3
:1004430074FF13FC7D80E480EFC0E0EFFBEEFAED78
:10045300F9ECF8120169D0E0F5F0EFFBEEFAEDF9F3
:10046300ECF8120997A3A3A3A3E8C0E0E9C0E0EA6C
:10047300C0E0EBC0E0C0F01201691209B4A3A3A36A
:10048300A3120078D0F0D0E0FBD0E0FAD0E0F9D0AE
:10049300E0F8D5F0D4223F8000004120000042C89C
:1004A3000000447A0000461C400047C350004974D2
:1004B30024004B1896804CBEBC205A0E1BCA6753AF
:1004C300C21C749DC5AEFB60065407601C23231237
:1004D30004F7EB543860091204E31204F2120169C1
:1004E300ECF8EDF9EEFAEFCB22EB1204F280F154C3
:1004F3003803241C900499FE93FC0EEE93FD0EEE3C
:10050300930ECE93FF22F920E72824F950037907AD
:10051300E4F42402FB18DBFDE624FB5014E9600D30
:10052300E4F618E604F6B40A08E4F6D9F57401F61D
:100533000A22C2D522ED33EC3392D5FA602AB4FFF6
:1005430033EDC2E77BFF60067A05795DE4227A0525
:10055300796620D5047A057961224E614E002B49D4
:100563004E46002D494E4600E47A08F608DAFC7B35
:1005730000740722E8C0E0ECC0E0EDC0E0EEC0E0AC
:10058300EFC0E0EA75F010A4CAABF075F04DA42BF0
:10059300FBE435F0FCEA2410FAEB34C5FBEC34D968
:1005A300FCEDC2E7FF75F056A4F42411C5F0F43452
:1005B300C58FF0A42AE5F03BE43CF620E7141204CF
:1005C300C9D0E0FFD0E0FED0E0FDD0E0FC12027223
:1005D3008014F4041204C9D0E0FFD0E0FED0E0FDA3
:1005E300D0E0FC120169D0E0F8E6FAEDD2E7CD33B2
:1005F300EC332482FBE4C3CF33CFCE33CECD33CD24
:1006030033DBF37B0775F00A846004F6081B0AE505
:10061300F0F6088FF0740AA4FFACF08EF0740AA40D
:100623002CFEACF050010C8DF0740AA42CFDE435C3
:10063300F0F608DBDE740722E709F608DFFA8046E6
:10064300E709F208DFFA803E88828C83E709F0A38A
:10065300DFFA8032E309F608DFFA8078E309F2086B
:10066300DFFA807088828C83E309F0A3DFFA806469
:1006730089828A83E0A3F608DFFA805889828A8315
:10068300E0A3F208DFFA804C80D280FA80C680D4DF
:10069300806980F28033801080A680EA809A80A8E7
:1006A30080DA80E280CA803389828A83ECFAE49319
:1006B300A3C8C582C8CCC583CCF0A3C8C582C8CCA7
:1006C300C583CCDFE9DEE7800D89828A83E493A3C7
:1006D300F608DFF9ECFAA9F0EDFB2289828A83ECB4
:1006E300FAE0A3C8C582C8CCC583CCF0A3C8C58231
:1006F300C8CCC583CCDFEADEE880DB89828A83E469
:1007030093A3F208DFF980CC88F0EF60010E4E600E
:10071300C388F0ED2402B4040050B9F582EB24023F
:10072300B4040050AF232345822390068B73BB018F
:100733000689828A83E0225002E722BBFE02E3227B
:1007430089828A83E49322BB010CE58229F582E541
:10075300833AF583E0225006E92582F8E622BBFEC0
:1007630006E92582F8E222E58229F582E5833AF556
:1007730083E49322BB010689828A83F0225002F725
:1007830022BBFE01F322EF8DF0A4A8F0CF8CF0A4DE
:1007930028CE8DF0A42EFE22BC000BBE0029EF8DC7
:1007A300F084FFADF022E4CCF875F008EF2FFFEEF4
:1007B30033FEEC33FCEE9DEC984005FCEE9DFE0F02
:1007C300D5F0E9E4CEFD22EDF8F5F0EE8420D21C5D
:1007D300FEADF075F008EF2FFFED33FD40079850A5
:1007E30006D5F0F222C398FD0FD5F0EA22C2D5EC6C
:1007F30030E709B2D5E4C39DFDE49CFCEE30E71578
:10080300B2D5E4C39FFFE49EFE12079BC3E49DFDA4
:10081300E49CFC800312079B30D507C3E49FFFE4ED
:100823009EFE22A3F8E0C5F025F0F0E58215827064
:10083300021583E0C838F0E822E88FF0A4CC8BF0EF
:10084300A42CFCE98EF0A42CFC8AF0EDA42CFCEA89
:100853008EF0A4CDA8F08BF0A42DCC3825F0FDE9C3
:100863008FF0A42CCD35F0FCEB8EF0A4FEA9F0EBB9
:100873008FF0A4CFC5F02ECD39FEE43CFCEAA42DC5
:10088300CE35F0FDE43CFC2275F008758200EF2FB5
:10089300FFEE33FECD33CDCC33CCC58233C5829B43
:1008A300ED9AEC99E58298400CF582EE9BFEED9A69
:1008B300FDEC99FC0FD5F0D6E4CEFBE4CDFAE4CC05
:1008C300F9A88222B800C1B90059BA002DEC8BF007
:1008D30084CFCECDFCE5F0CBF97818EF2FFFEE33C4
:1008E300FEED33FDEC33FCEB33FB10D703994004EF
:1008F300EB99FB0FD8E5E4F9FA227818EF2FFFEE16
:1009030033FEED33FDEC33FCC933C910D7059BE946
:100913009A4007EC9BFCE99AF90FD8E0E4C9FAE4A2
:10092300CCFB2275F010EF2FFFEE33FEED33FDCC41
:1009330033CCC833C810D7079BEC9AE899400AED2B
:100943009BFDEC9AFCE899F80FD5F0DAE4CDFBE4D3
:10095300CCFAE4C8F922C3E49FFFE49EFEE49DFDC4
:10096300E49CFC22EB9FF5F0EA9E42F0E99D42F005
:10097300E89C45F022E8600FECC313FCED13FDEE99
:1009830013FEEF13FFD8F122E6FC08E6FD08E6FEAE
:1009930008E6FF22E493FC740193FD740293FE7452
:1009A3000393FF22E6FB08E6F908E6FA08E6CBF82C
:1009B30022E493F8740193F9740293FA740393FB9A
:1009C30022ECF608EDF608EEF608EFF622ECF0A3BB
:1009D300EDF0A3EEF0A3EFF022A42582F582E5F07B
:1009E3003583F58322FAE6FB0808E6F925F0F618C5
:1009F300E6CA3AF622D083D082F8E49370127401E7
:100A030093700DA3A393F8740193F5828883E47321
:100A13007402936860EFA3A3A380DF8A838982E4CF
:100A230073EF4E6012EF60010EEDBB010B89828AFA
:100A330083F0A3DFFCDEFA2289F05007F709DFFC1D
:100A4300A9F022BBFEFCF309DFFCA9F022E5602438
:100A53004CF8E60560227849302F02784CE475F0B3
:100A6300011209E80207312028EB7F2ED2288018D3
:100A7300EF540F2490D43440D4FF302C0BEF24BF19
:100A8300B41A0050032461FFE56160021561056437
:100A9300E56470020563302F0D7849E475F00112A7
:100AA30009E8EF0207770219EB7403D22F8003E4FE
:100AB300C22FF5608B498A4A894BE4F561F563F5EA
:100AC30064E56160077F20120A8B80F57562FFC2BF
:100AD30029C228C22AC22BC22DC22EC230120A59E1
:100AE300FF700D302F057F00120A9CAF64AE6322A6
:100AF300B4255FC2D5C22C120A59FF24D0B40A0010
:100B0300501A75F00A786130D50508B6FF0106C69C
:100B1300A426F620D5047002D22B80D924CFB41A90
:100B230000EF5004C2E5D22C020D89D22980C6D22F
:100B33002880C0D22A80BCD2D580BAD22D80B47F7F
:100B430020120A8B202A077401B5610040F1120AB2
:100B530050FF120A8B020AC4D230D22E8095120A99
:100B630050FB120A50FA120A50F94A4B7006798068
:100B73007A0E7BFF202A2EE561602A7E008E827525
:100B8300830012074A60060EEE656270F0C2D5EB71
:100B9300C0E0EAC0E0E9C0E0EE120DE9D0E0F9D030
:100BA300E0FAD0E0FB120731FF60AAEBC0E0EAC035
:100BB300E0E9C0E0120A8BD0E02401F9D0E0340070
:100BC300FAD0E0FBE5620460DCD562D98087D22AE3
:100BD30080A2120DCC60F7E562700104120509A929
:100BE30062600DE562600914F562120E73EF60F343
:100BF300EA30E702F404C3995077EAF4256204303B
:100C0300E701E404F562800D120DCC60C1EA0562D0
:100C13002562120509EA785FF630E701E4256204EC
:100C2300D56204202D0114120DE9E4C0E0120E7305
:100C3300785FE6601320E70714F6120A7380220434
:100C4300F6D0E014C0E07F00120A73E56260071279
:100C53000A6A1562800B302D03120A6AD0E0020A79
:100C6300C4D0E00480C5120DCC60A0E56204120577
:100C730009785FEAF6E562202D026001042404127C
:100C83000DE974FF04C0E0120E73120A73E56220CB
:100C93002D026003120A6AD0E0B562E87F45120AAA
:100CA3007D785FE67F2B30E7047F2DF404C0E012EC
:100CB3000A8BD0E075F00A84C0F0120A74D0E012F7
:100CC3000A74020AC4791080027908C22EC23080E5
:100CD30008D2D5790A8004790AC2D5E56204700284
:100CE300F562E4FAFDFEFF120A50FC7B082029138B
:100CF300120A50FD7B1030280A120A50FE120A50C5
:100D0300FF7B20EC3382D592D55013C3E430280601
:100D13009FFFE49EFEE42029039DFDE49CFCE4CBBD
:100D2300F8C229EC700CCFCECDCCE824F8F870F3E0
:100D33008017C3EF33FFEE33FEED33FDEC33FCEBF3
:100D430033FB994002FB0FD8E9EB302905F8D0E0DB
:100D5300C448B229C0E00AEC4D4E4F78207B0070A6
:100D6300C2EAB5620040BCC0E0120DEBD0F0D0E0A7
:100D7300202904C4C0E0C4B229C0F0120A74D0F020
:100D8300D5F0EB020AC41209F80B61530CC8580BD7
:100D9300324C0B2E420CCC4F0CD4440CD4490B4791
:100DA300430CDA550C0B460C69450BD5470EA05086
:100DB3000B362D0B3A2E0B5D2B0B3E230B5B200EBC
:100DC300892A0AF64800000B55E562B4FF037562F1
:100DD30006120A50FC120A50FD120A50FE120A5063
:100DE300FF7858020538790AA2D5202B14302D0933
:100DF300B910020404B9080104A2D5202E0250013F
:100E030004202A68922AB561005034C0E07F203064
:100E13002B197F30A22A722E722D500F120E42C24E
:100E23002AC22EC22DC2307F30800F302D03E9C07D
:100E3300E0120A8B302D03D0E0F9D0E0B561CC305D
:100E43002D177F30B9100C120A8B7F58302C077F77
:100E5300788003B90803120A8B302A057F2D020A12
:100E63008B7F202030F87F2B202EF322922A80CFF5
:100E73007F00B4070050052458F8E6FF22286E755A
:100E83006C6C2900D229120A503029F8C2297861E2
:100E930030D50108F6020AF62D50434958120A507C
:100EA3002403B405004001E4900E9B93120A7C7462
:100EB3003A120A7CD22B756104020CC825730020F8
:100EC3002573003E005F2573002020202020202072
:100ED3002020202020202020004B4D480025337562
:100EE300004D5048003C005F257320202020202027
:100EF300202020202020002530337520004C415431
:100F03005F3A5F25635F25303375405F2530322EAE
:100F13003032662720004C4F4E5F3A5F25635F25D2
:100F2300303375405F2530322E303266272000443F
:100F330049525F3A5F2530337540002533627500AF
:100F43005E0025733A2025362E3166204D69002533
:100F5300733A2025362E3166204B4D0025733A20F7
:100F6300252D322E316600560025733A20256278EE
:100F73002E253162780025733A20002562752F25CE
:100F830062752F25347500204B204D204820284BB7
:100F93004D2F482900204D2050204820284D494CF2
:100FA300452F482900474D5420202B2562642000FB
:100FB300474D54202025626420200025735F25734C
:100FC3000053454C455A494F4E455F4D4F444F20C2
:100FD3002020004C494D495445202020202020202A
:100FE300202020200050554E54495F5554454E54FF
:100FF30049202020202000494C4C554D494E415A50
:10100300494F4E4520202020004D49535552415F02
:101013005041455345202020202000494E464F5F34
:1010230044454C5F53495354454D41200020554E90
:1010330049546D2020202020202020202000205AE9
:101043004F4E415F44495F54454D504F202000208F
:1010530053554F5F44495F43414D50414E4120003A
:10106300FF648AFF660EFF585AFF7197FF624AFFBB
:101073003C66FF656AFF726CFF67970122000120DF
:10108300000123000121004188100044880600006C
:101093000000418811004188040041880F00418805
:1010A3000D004188050041880200418621004185E9
:1010B3001F0041852000448737000000004A874D08
:1010C300000000000000000000004A874300000009
:1010D3000000000000000044872D0000000042874C
:1010E3002B00004487330000000041873100418713
:1010F3005D0042872000004187320042875B1C204D
:10110300448722000000004187290041872A0041CB
:1011130087280044875E0000000041876300418701
:101123006400418762004487570000000044871C25
:101133000000000044873F00000000418726004173
:101143008727004A87920000000000000000FF008C
:101153004A879C0000000000000000FF004287A6B1
:1011630000004287B600004E87A800000000000080
:1011730000000000000000004187B9004187B8006B
:101183004A88230000000000000000FF0042882D71
:1011930000004A882F0000000000000000FF00420A
:1011A300883900004987C7000502010504020506C6
:1011B3004987BE0005020105040205064187D100E7
:1011C3004187D0004287D200004187D4005687D799
:1011D30000000000560000000000000000000000B6
:1011E30000FF0000000002A4862202A686224C878C
:1011F300F51F1C1F1E1F1E1F1F1E1F1E1F41841BAA
:101203000002A8000041883B0041883CFF01AA007E
:1012130041883D0041883F0041883E000124000091
:1012230025730025336275005E004E452533750036
:101233004520253375005345253375005320253349
:10124300752A00534F253375004F20253375004E03
:101253004F253375004E202533750025336C7500FB
:101263004D00202020203E002020203E3E00202054
:101273003E3E3E00203E3E3E3E003E3E3E3E3E0063
:1012830025732020200025733E20200025733E3E39
:10129300200025733E3E3E00253475004D50480026
:1012A3004B4D48004E452533754000452025337589
:1012B30040005345253375400053202533754000C6
:1012C300534F25337540004F2025337540004E4F53
:1012D30025337540004E2025337540002020202003
:1012E30020400025352E3166204D690025352E31ED
:1012F30066204B4D00253262753A25303262750007
:101303002573253262753A2530326275007E0025D9
:10131300362E3166204D690025362E3166204B4D21
:1013230000253375204D504800253375204B4D481B
:101333000025342E3166204D50480025342E316669
:10134300204B4D4800253262752F253262750025EA
:10135300733A252D322E316656004241540025350D
:101363002E31664D690025352E31664B4D002533F0
:10137300754D5048002533754B4D48002533750096
:1013830025735F4445002532750044495F2573008A
:101393005175696E74657A7A00414C4552544552D1
:1013A30000475053202573002573202573202120E7
:1013B30020003A70FA83BCAAE9E43E81E0F8BF9DBD
:1013C300E9E63F80000039283C1ABB9969663DA3D2
:1013D30035E3BF255DE73FC90FDB418DDBCCC44956
:1013E30036EE45C9913FC5B0F83D3F800000C317B5
:1013F300F534452FFA73C60AFDDD1214A404A2E1E5
:1014030092281420E0159013B5740412044C80261E
:101413001214A430E102B22820E0EB8C278D288E31
:10142300298F2A9013C9740412044CA827A928AA47
:1014330029AB2A120169ED4C6007302804EC648063
:10144300FC221214A4C0E08C278D288E298F2A90A9
:1014530013ED740312044CA827A928AA29AB2A1256
:101463000169ECC527FCEDC528FDEEC529FEEFC5D6
:101473002AFF9013DD740312044CD082A827A928F5
:10148300AA29AB2AE58230E007120272B22880A6AD
:10149300EFCBFFEECAFEEDC9FDECC8FC1202728071
:1014A30095ED33EC547FCC33922824605007D0E081
:1014B300D0E00204377B837AF97922783E120169FE
:1014C300EDF933ECF83324815011EFFBEEFA1203FC
:1014D300CB12038DECB2E7FC120078ED33EC3360F2
:1014E3002F2403F8C313FCED92E7FDE82481E450B5
:1014F3001FECF8EDF9EEFAEFFB1203CBEF04C2E0B9
:10150300FCF582120397ECB2E7FC120078E5820344
:10151300FAED33EC3360071413FCED92E7FDEA2296
:10152300BE1249253E4CCCCDBEAAAAAB3F800000DB
:101533003E7ADBB03EED63383F24BC7D3F490FDB91
:10154300ED33ECC2E7CC339228B4FF13ED547F6044
:10155300030204377FDB7E0F7DC97C3F02163EC248
:1015630029C3947F401E7007EDD2E794904015EF96
:10157300FBEEFAEDF9ECF87F007E007D807C3F12F4
:101583000272D229ED33EC33248430E705E4C0E062
:10159300806D04FAEDD2E754F0C333DAFD54073417
:1015A300002323C0E0CCC0E0F8EDC0E0F9EEC0E0DA
:1015B300FAEFC0E0FBE4120397EC24FEFC8C388DB9
:1015C300398E3A8F3B1201697B007A007980783F2C
:1015D300120078ECC538B2E7FCEDC539FDEEC53A2B
:1015E300FEEFC53BFFD0E0FBD0E0FAD0E0F9D0E05E
:1015F300F8120078A838A939AA3AAB3B1202728CC8
:10160300388D398E3A8F3B901523740312044CA8FE
:1016130038A939AA3AAB3B120169D0E0600F242FF5
:10162300F582E43415F5831209B412007830290BDE
:101633007BDB7A0F79C978BF120078ED33EC336026
:1016430006ECA22892E7FC22C229C22AC22BC22C92
:10165300F9E4F52EF52FFCFDFEFFE91028EA202B17
:101663000CB42D04D22BD322B42B02D32224D0507A
:101673004794095041240A302C15F8852FF0740A39
:10168300A42872E74051C5F0704D85F02FD322D2C4
:101693002AC0E0E4FBFA79207841120169ECF8ED05
:1016A300F9EEFAEFFBD0E0FCE41203971200783076
:1016B30029B4152ED322240A202C20B4FE07202976
:1016C3001AD229D32224EB600424E0700EA22B92B9
:1016D30029D22CC22BD322C3020437E4302C0BE5CE
:1016E3002F302B02F404A229922B302AEA252E2034
:1016F300D2E5A2E7922C5002F404B4260050D8CCD1
:10170300C0E0EDC0E0EEC0E0EFC0E0EC1204C9D0F1
:10171300E0FFD0E0FED0E0FDD0E0FC202C0512017C
:10172300698003120272302B0312037CC32202046A
:101733003722EDA2E7D2E7F9EC3340F260F3B4FFCE
:1017430008ED547F70E8020441F82481C2E0C0E050
:10175300F40428FAC313FCED92E7FD8C308D318E2F
:10176300328F33EEA2E7E9BA7F02C3133400940049
:10177300FA75F091A4E5F013F494FE8AF0A433E52E
:10178300F033248CD313FDE492E7FE7F007C3F7596
:101793008302ECC0E0F8EDC0E0F9EEC0E0FAEFC080
:1017A300E0FBAC30AD31AE32AF33120272D0E0FBAE
:1017B300D0E0FAD0E0F9D0E0F8120078ED6480FDD3
:1017C30030E7011CD583CBED33CC33F8D0E0A2E76F
:1017D3001328C313CC13FD227581AA02181C0231EE
:1017E30037E493A3F8E493A34003F68001F208DF00
:1017F300F48029E493A3F85407240CC8C333C454D6
:101803000F4420C8834004F456800146F6DFE48089
:101813000B010204081020408090107EE47E0193A7
:1018230060BCA3FF543F30E509541FFEE493A3605B
:10183300010ECF54C025E060A840B8E493A3FAE4B6
:1018430093A3F8E493A3C8C582C8CAC583CAF0A307
:10185300C8C582C8CAC583CADFE9DEE780BE8F3345
:101863008E328D318C30AB37AA36A935A8341202AB
:10187300721215438F338E328D318C30E53430E75D
:1018830047ECC0E0EDC0E0EEC0E0EFC0E0E4FFFEF7
:10189300FDFCAB33AA32A931A83012030F7BDB6006
:1018A3000250087A0F7949784080067A0F7949788F
:1018B300C0D0E0FFD0E0FED0E0FDD0E0FC12007825
:1018C3008F338E328D318C30AF33AE32AD31AC309D
:1018D300228B278A288929AB2AAA2BA92C12073104
:1018E300FEAB27AA28A929120731FF6E702BEF60E0
:1018F3000DE52E152E7002152D14452D70037F0056
:101903002274012529F529E43528F5287401252CAD
:10191300F52CE4352BF52B80BEAB27AA28A9291279
:101923000731FFD3EE6480F8EF64809840037F01B2
:10193300227FFF22D2288B2B8A2C892D121973C068
:10194300E0FF121A12D0E040F312165E400122ECBF
:10195300C0E0EDC0E0EEC0E0EFC0E0121973D0F0DC
:10196300AFF0D0F0AEF0D0F0ADF0D0F0ACF080D965
:10197300E475F001782B1209E8020731257300534F
:1019830050454544005253002533754D50480025BA
:1019930033754B4D48004C41534552003E3E3E008B
:1019A3004B412042414E4400256264004B2042419A
:1019B3004E4400582042414E440085434C85444DDB
:1019C30085454EEBC546FBEAC547FAE9C548F97FAD
:1019D30009784F120731F60809E970010ADFF4AB01
:1019E30046AA47A948020AACEFB40A07740D1219B4
:1019F300F6740A309811A899B8130CC2983098FD60
:101A0300A899C298B811F63099FDC299F59922EFB9
:101A1300C394094005EF940E4003BF2003D3800114
:101A2300C3222533750025730025733100257332D6
:101A33000025730025733A2575005F564F4C554DAD
:101A43004520202020202020202000434F4C4C45BF
:101A5300474152455F4750530056454C4F43495405
:101A63002E00414C4C41524D450041434345534F99
:101A7300202020202000444953434F4E4E455353CA
:101A83004F0043414D455241004249444952455A52
:101A93002E0044492053545241444100434F4E5475
:101AA300524F4C4C4F0053434F504F20444900502A
:101AB300455249434F4C4F534F00504F53495A4996
:101AC3004F4E45004156564552542E005554454EEF
:101AD3005445005F504F53544F0041474749554EBB
:101AE300544F005049454E4F00454C494D494E41D6
:101AF300544F0056554F544F004D454E555F50526D
:101B0300494E434950414C45005F53454C455A4962
:101B13004F4E455F4D4F444F2020004C494D495493
:101B230045005F494C4C554D494E415A494F4E452E
:101B3300202020004D49535552415F5041455345A4
:101B43002020202000494E464F5F44454C5F5349B7
:101B53005354454D4120005F554E49546D2020207C
:101B63002020202020202020005A4F4E415F44494E
:101B73005F54454D504F0053554F0053554F5F44ED
:101B8300495F43414D50414E41202020005553456C
:101B93005220494E464F0052495052495354494EE0
:101BA3004900545241474954005354414E44415211
:101BB30044005041525449434F4C41524900434F12
:101BC3004D4F4449546D00534920004E4F4E00423F
:101BD3005553534F4C41004F444F0044415441002F
:101BE300546563686E6F6C6F676961004155544F4C
:101BF3002D54455354004E455353554E20444154A0
:101C030049004241545445524941005452495020DD
:101C130054494D4500534F465457415245004441A2
:101C2300544920202020004D454D4F52495A5A41D6
:101C330054410050554E5449205554454E54490083
:101C4300522F4F444F004D4544494F0054454D508A
:101C53002E0000000000000000004F4F00000006AF
:101C63000006000000487A410000F8252524F8000A
:101C7300007F25251A007D4140417D000000000BB7
:101C8300070000487A490000F824252525F80303B6
:101C93000000000008083E08080000000058380053
:101CA300080808080800000040000000201008048D
:101CB30002003E5149453E0000427F400000426120
:101CC300514946002241494936001814127F100039
:101CD3002745454539003C4A49493000017109050A
:101CE3000300364949493600064949291E00003692
:101CF30036000000005B3B00000000081C3E7F0034
:101D03001414141414007F3E1C0800000201590926
:101D13000600324959413E007E1111117E00417F78
:101D2300494936003E4141412200417F41413E0045
:101D33007F49494141007F09090901003E41494961
:101D43007A007F0808087F0000417F41000020409F
:101D5300413F01007F08142241007F404040400082
:101D63007F020C027F007F0204087F003E41414155
:101D73003E007F09090906003E4151215E007F09AB
:101D83001929460026494949320001017F01010012
:101D93003F4040403F000718601807003F4038406D
:101DA3003F006314081463000708700807006151BB
:101DB30049454300007F4141000002040810200010
:101DC3000041417F00000402010204004040404002
:101DD30040000004020100002054545478007F485E
:101DE30044443800384444442000384444487F0085
:101DF300385454540800087E09020000081454544F
:101E03003C007F080404780000447D40000020402B
:101E1300443D0000007F1028440000417F40000043
:101E23007804180478007C08040478003844444497
:101E330038007C14242418001824147C4000007CEF
:101E430008040400485454542000043E4420000075
:101E53003C4040207C001C2040201C003C40304083
:101E63003C004428102844004C5050503C0044642B
:101E7300544C440000083641000000007700000085
:101E83000041360800000804081008002A552A55A6
:101E93002A0008000000000000000000000000000D
:101EA3000000000400F8F800000D0D0006383800AB
:101EB3003838000000000000000820F8F820F8F887
:101EC3002000020F0F020F0F0200003078CE8E1891
:101ED300100000040C38390F060008183C24BCD845
:101EE3006030000006030E1E121E0C0800B0F848F6
:101EF3007830000000070F0809070F09023838007F
:101F03000004E0F81C04030F1C1004041CF8E01088
:101F13001C0F030780A0E0C0E0A0800002030103C0
:101F23000200068080E0E0808000000303000003DD
:101F33000000002C3C1C0680808080808000000014
:101F43000000000400000000000C0C00060000C0AC
:101F5300F03C0C0C0F030000000800F0F80868F8D0
:101F6300F00000070F0B080F07000800202030F8CF
:101F7300F80000000000000F0F00000800303808D0
:101F830088F87000000C0E0B0908080008003038B0
:101F93008888F8700000060E08080F070008000084
:101FA300F8F800E0E00000030302020F0F0208004C
:101FB300F8F88888880800000808080C0703000858
:101FC30000C0E07858C8800000070F08080F07001A
:101FD3000800080888E878180000000E0F010000C8
:101FE30000080070F8C888F8700000070F08090F90
:101FF30007000800F0F80808F8F0000000090D0FCA
:102003000301000800000060600000000000000CF5
:102013000C000000080000006060000000000000E9
:102023002C1C000000070080C0E0F0F80000000155
:1020330003070F000560606060000C0C0C0C0007C8
:1020430000F8F0E0C08000000F0703010000076004
:10205300701090F0600000001B1B000000040038AB
:102063002838000000000800E0F01818F0E0000035
:102073000F0F01010F0F000800F8F88888F87000AF
:10208300000F0F08080F07000800F0F808083830A1
:102093000000070F08080E06000800F8F80818F0FB
:1020A300E000000F0F080C0703000800F8F8888809
:1020B300880800000F0F08080808000800F8F888CF
:1020C30088880800000F0F00000000000800F0F8E7
:1020D300080838300000070F08090F0F000800F840
:1020E300F88080F8F800000F0F00000F0F000800C1
:1020F3000008F8F80800000000080F0F08000008A7
:102103000000000000F8F80000060E08080F0700A2
:102113000800F8F880E0781800000F0F00030F0C98
:10212300000800F8F80000000000000F0F0808087E
:1021330008000800F8F820C020F8F8000F0F00018D
:10214300000F0F0800F8F860C080F8F8000F0F00C8
:1021530000010F0F0800F0F80808F8F00000070F5F
:1021630008080F07000800F8F88888F87000000FC7
:102173000F00000000000800F0F80808F8F0000065
:10218300070F08181F17000800F8F88888F8700070
:10219300000F0F00010F0E0008003078C8881810D8
:1021A3000000040C08090F060008000808F8F808E6
:1021B30008000000000F0F0000000800F8F80000FE
:1021C300F8F80000070F08080F07000800F8F800E8
:1021D30000F8F8000003070C0C0703000800F8F8E8
:1021E30000C000F8F800010F0E010E0F01080018DF
:1021F30038E0C0381800000E0F00010F0E00080071
:1022030078F88080F878000000000F0F00000008C5
:1022130000080888C8783800000E0F09080808006D
:102223000404FCFC00101F1F000638F8C000000067
:102233000000030F0C0004FCFC04001F1F10000827
:102243000C1E92DE6C301800000301060F090F0606
:102253000400000000000000000400000000000073
:1022630000000800F2FA1818FAF200000F0F01013B
:102273000F0F000800FAFA0000FAFA0000070F0C2B
:102283000C0F07000800F2FA0808FAF20000070F23
:1022930008080F07000800F0FA1A19F9F000000FF8
:1022A3000F01010F0F000800F8FA8A89890800005E
:1022B3000F0F08080808000800080AFAF9090800BF
:1022C3000008080F0F0808000800F0FA0A09F9F0DF
:1022D3000000070F08080F07000800F8FA0201F9C9
:1022E300F80000070F08080F07000800FAF9C38277
:1022F300F9F800000F0F00010F0F000800F8FA01B2
:1023030001FAF80000070F0C0C0F07000800F8F99A
:10231300898A8A0800000F0F0808080800080008C7
:1023230009F9FA0A08000008080F0F080800080056
:10233300F0F9898AFAF000000F0F01010F0F00086E
:1023430000F8044444788000000F000202020100F8
:102353000800C0E02020E0C00000070F08080F07B6
:10236300000800E0E02020E0C000003F3F08080F25
:1023730007000800C0E02020E0E00000070F080885
:102383003F3F000800E0E08040606000000F0F0066
:10239300000000000800C0E0202020200000080901
:1023A30009090F0600080020F8F82020200000008B
:1023B300070F080808000800E0E00000E0E0000064
:1023C300070F08080F0F000800E0E00000E0E0003E
:1023D3000003070C0C0703000800E0E000C000E066
:1023E300E000030F0C030C0F03080060E08080E0A3
:1023F3006000000C0E03030E0C000800E0E0000078
:10240300E0E000002327341C0F03000800F9F98AD9
:102413008A8A0800000F0F0808080800FF1E95FFAE
:102423001EA6FF1EAFFF1EBCFF1ECDFF1EDDFF1E3F
:10243300EEFF1EFFFF1F04FF1F0DFF1F16FF1F25CB
:10244300FF1F32FF1F39FF1F46FF1F4FFF1F5CFF98
:102453001F6DFF1F7EFF1F8FFF1FA0FF1FB1FF1FF9
:10246300C2FF1FD3FF1FE4FF1FF5FF2006FF201746
:10247300FF2028FF2037FF2042FF2051FF2060FF6D
:102483002069FF207AFF208BFF209CFF20ADFF20D7
:10249300BEFF20CFFF20E0FF20F1FF2102FF211329
:1024A300FF2124FF2135FF2146FF2157FF2168FF2C
:1024B3002179FF218AFF219BFF21ACFF21BDFF2151
:1024C300CEFF21DFFF21F0FF2201FF2212FF222393
:1024D300FF222CFF2239FF2242FF2253FF225CFFFF
:1024E3002265FF2276FF2287FF2298FF22A9FF227F
:1024F300BAFF22CBFF22DCFF22EDFF22FEFF230FD8
:10250300FF2320FF2331FF2342FF2353FF2364FFD5
:102513002375FF2386FF2397FF23A8FF23B9FF23F8
:10252300CAFF23DBFF23ECFF23FDFF240E0CF0F88F
:10253300FCFEFE0E8EFEFEFCF8F0FFFFFFFFFFF831
:102543001FFFFFFFFFFF0F1F3F7F7F70707F7F3FE6
:102553001F0F0C000070707078FCFCFEFEFE000084
:102563000000000000FFFFFFFFFF0000000000006D
:10257300007F7F7F7F7F000C00F0FCFCFE0E0EFED1
:10258300FEFCF8F000000080E0F8FEFFFF3F1F03B1
:1025930000787E7F7F7F7F73707070000CF0FCFC8F
:1025A300FEFE0E0EFEFEFCFCF0C1C1C1C1DD1C3CF3
:1025B300FFFFFFF7E30F3F3F7F7F70707F7F3F3F5A
:1025C3000F0C000080F0FE3EFEFEFEFE0000E0FC6D
:1025D300FFDFC3C0FFFFFFFFC0C0070707070707F1
:1025E3007F7F7F7F07070CFEFEFEFEFE0E8E8E8E24
:1025F3008E0E0E8F8F8F8F8F0303FFFFFFFFFE0F54
:102603003F3F7F7F70707F7F3F3F0F0CF0F8FCFEF2
:10261300FE0E0E7E7E7C7C70FFFFFFFFFF0607FF32
:10262300FFFFFEFC0F3F3F7F7F70707F7F3F3F0FB9
:102633000C001E1E1E1E1E1EFEFEFEFEFE000000E1
:1026430000E0F8FFFFFF1F07000060787F7F7F1F18
:1026530007000000000CF0FCFCFEFE0E0EFEFEFC6C
:10266300FCF0E3F7FFFFFF1C1CFFFFFFF7E30F3F47
:102673003F7F7F70707F7F3F3F0F0CF0FCFCFEFEBF
:102683000E0EFEFEFCF8F03F7FFFFFFFE060FFFF52
:10269300FFFFFF0E3E3E7E7E70707F7F3F1F0F0267
:1026A300707000000E0E020C040CFEFEFCF8F0E04D
:1026B300C08000000000FFFFFFFFFFFFFFFFFF7E62
:1026C3003C187F7F3F1F0F070301000000000E042B
:1026D3000C1E1E0C00000000000000000E00C0FED7
:1026E300FEFEFE1EFEFEFEFEC00000E0FFFFFFFF3B
:1026F300878087FFFFFFFFE0007F7F7F7F0707075C
:1027030007077F7F7F7F000CFEFEFEFEFE1E1EFE80
:10271300FEFCFCF0FFFFFFFFFF1E1EFFFFFBFBF1B4
:102723007F7F7F7F7F78787F7F7F3F1F0D0CFEFE4B
:10273300FEFEFE1E1EFEFEFCFCF8FFFFFFFFFF0079
:1027430000FFFFFFFFFF7F7F7F7F7F78787F7F7FA3
:102753003F1F0BFEFEFEFEFE1E1E1E1E1E1EFFFF65
:10276300FFFFFF3C3C3C3C3C007F7F7F7F7F7878D2
:10277300787878780B0C0D05080DFEFEFEFEFE0042
:10278300C0F8FEFEFE3E06FFFFFFFFFF7FFFFFFFD9
:10279300F78000007F7F7F7F7F00030F7F7F7F7C39
:1027A300700AFEFEFEFEFE0000000000FFFFFFFFBA
:1027B300FF00000000007F7F7F7F7F787878787844
:1027C300110CFEFEFEFEF88000FEFEFEFEFEFFFF85
:1027D300FFFFFF1FF8FFFFFFFFFF7F7F7F7F7F006C
:1027E300011F7F7F7F7F0CF0F8FCFEFE1E1EFEFEA6
:1027F300FCF8F0FFFFFFFFFF0000FFFFFFFFFF0FED
:102803001F3F7F7F78787F7F3F1F0F0C0C0CFEFEEE
:10281300FEFEFE1E1EFEFEFEFCF8FFFFFFFFFF1E78
:102823001EFFFFFFF7E37F7F7F7F7F00007F7F7FB8
:102833007F7F0DF0FCFCFEFE1E1EFEFEFCFCF8007E
:1028430083878F9F9F3F7F7EFCF8F8F0C00F1F3F69
:102853007F7F7878787F7F3F3F0F0C1E1E1EFEFE22
:10286300FEFEFEFE1E1E1E000000FFFFFFFFFFFF19
:102873000000000000007F7F7F7F7F7F0000000C4F
:102883000F151EFEFEFEFEC00000FEFEFEFEFE0055
:1028930000C0FEFEFEFE1E001FFFFFFFFF00FFFF46
:1028A300FF03FFFFFF00FFFFFFFF1F0000001F7F6D
:1028B3007F7F7E7F7F0100017F7F7C7F7F7F1F0083
:1028C300000D063EFEFEF8E000C0F8FEFE3E0600E8
:1028D30000C0FFFFFF3FFFFFFFC00000707E7F7F50
:1028E3001F0100011F7F7F7E700D0A001E1E1EDE6A
:1028F300FEFEFEFE7E0080F0FEFFFFFF1F0300785A
:102903007F7F7F7F7F78787878FF2530FF2555FF9D
:10291300257AFF259FFF25C4FF25E9FF260EFF2605
:1029230033FF2658FF267DFF26A2FF26A9FF26AAEE
:10293300FF26ABFF26ACFF26D1FF26D2FF26DFFF03
:10294300270AFF272FFF2730FF2755FF2777FF276A
:1029530078FF2779FF277AFF277BFF277CFF27A4B0
:10296300FF27C3FF27C4FF27E9FF280EFF280FFF18
:102973002810FF2835FF285DFF2882FF2883FF28C2
:1029830084FF28C4FF28ECFF28ED0B013C242424FA
:1029930024242424243C000B013C3C3C3C3C3C3C94
:1029A3003C3C3C000A0200FE020202020202FE005C
:1029B300007F4040404040407F000A0200FEFEFE90
:1029C300FEFEFEFEFE00007F7F7F7F7F7F7F7F0016
:1029D300100200000000C0F0FC1E1EFCF0C000004E
:1029E3000000C0F0FCFFFFFFFFC8C8FFFFFFFFFCB4
:1029F300F0C01E040000000000C0C0000018180052
:102A0300001F0204081F000018180000C0C00000C7
:102A130000008040404C8C000000000000000000DB
:102A2300000000000000000000000000CC4C40400B
:102A330003040464630000000000000000000000C1
:102A430000000000000000000000676505050000AD
:102A53000000000006060030300000B8A8A8E80017
:102A630000303000000606000000000010020000E5
:102A73000080E0F8FEFFFEF8E080000000006078D0
:102A83003E3F1F1F0F0F0F1F1F3F3E7860001002B6
:102A9300030F3EFEFCFCF8F8F0F0E0E0C0C080005D
:102AA30060783E3F1F1F0F0F07070303010100005C
:102AB3001002030F3EFEFCFCF8F8F8FCFCFE3E0F90
:102AC300030000000000030F3F7F3F0F03000000DF
:102AD3000000100280C0C0E0E0F0F0F8F8FCFCFE5B
:102AE3003E0F0300000101030307070F0F1F1F3FE2
:102AF3003E786000100200008080C0C0F0FCFFFF41
:102B0300FCF080000000030307070F0F0F1F1F1FB8
:102B13003F3F7F7C70801002C0C0E0E0F0F0F0F82F
:102B2300F8F8FCFCFE3E0E010000010103030F3F19
:102B3300FFFF3F0F010000001002010E3EFEFCFCF0
:102B4300F8F8F8F0F0F0E0E0C0C0000000010F3F3B
:102B5300FFFF3F0F0303010100001002000000808C
:102B6300F0FCFFFFFCF0C0C08080000000707C7FA1
:102B73003F3F1F1F1F0F0F0F070703032004000012
:102B83000000000000000080C0E0F0F8FCFEFCF84C
:102B9300F0E0C080000000000000000000000080A2
:102BA300C0E0F0F8FC1E1FFF0FFF03132B130303FA
:102BB30003030303FFFEFCF8F0E0C0800000000005
:102BC3000103070F1F3C7CF1F0F7E0E0E0E0E0E6F3
:102BD300E9E9E6E07F3F1F0F070301000000000063
:102BE30000000000000000000103070F1F3F1F0F3C
:102BF30007030100000000000000000000002004A3
:102C030000000000000000000080C0E0F0F8FCFEBF
:102C1300FCF8F0E0C08000000000000000000000AD
:102C23000080C0E0F0F8FC1E1F0FFF03132B1303FB
:102C33000303030303FF0F1E1CF8F0E0C080000032
:102C430000000103070F1F3C7CF0F7E0E0E0E0E049
:102C5300E6E9E9E6E0F7703C1C0F0703010000001A
:102C6300000000000000000000000103070F1F3FE9
:102C73001F0F070301000000000000000000000018
:102C8300200400000000000000000000000000C05D
:102C9300F0F8F8F0C00000000000000000000000A1
:102CA3000000000000000000000000C0F0FCFFFF77
:102CB30003030303FFFFFCF0C0000000000000005B
:102CC30000000000000000C0F0FCFFFFFFFFFFFF5B
:102CD30060606060FFFFFFFFFFFFFCF0C0000000CB
:102CE300000000000000070F0F0F0F0F0F0F0F0F53
:102CF3000C0C0C0C0F0F0F0F0F0F0F0F0F07000013
:102D030000001803FC02010101010181C1E1F1F995
:102D1300F9F1E1C181010101010102FCFF000000A1
:102D23000406070707FFFFFFFFFFFF070707060468
:102D3300000000FF3F40808080808080809F9F9FB5
:102D43009F9F9F80808080808080403F1803FC028B
:102D5300010101E1E1E1E1E1E1E1E1E1E161210120
:102D63000101010102FCFF00000000FFFF7F3F3F64
:102D73007FFFFFFFFCF8F0E0C080000000FF3F4052
:102D8300808080818080808080808183878F8F870F
:102D930083818080403F1803FC020101010101810E
:102DA300C1E1F1010101010101010101010102FC84
:102DB300FF0000183C7EFFFFFFFFFF7E7E7E7E7ECE
:102DC3007E7E7E7E7E0000FF3F408080808080810B
:102DD30083878F8080808080808080808080403F58
:102DE3001803FC020101010101010101010101F1CB
:102DF300E1C181010101010102FCFF00007E7E7E31
:102E03007E7E7E7E7E7E7EFFFFFFFFFF7E3C180080
:102E130000FF3F4080808080808080808080808F22
:102E23008783818080808080403F1803FC020101FA
:102E33000101012161E1E1E1E1E1E1E1E1E1E1013F
:102E4300010102FCFF00000080C0E0F0F8FCFFFF7E
:102E5300FF7F3F3F7FFFFF00000000FF3F40808078
:102E63008183878F8F87838180808080808081802A
:102E73008080403F07011C22514945221C30060037
:102E830000000000000080C0E0E0F0F8F8FC7C7E69
:102E93003E3E3E3E3F1F1F1F1F1E3E3E3E3E7C7C6E
:102EA300FCF8F8F0E0E0C080000000000000000043
:102EB30000C0F0F8FEFF7F3F0F0703010100000091
:102EC3000000000000000000000000000080C0E0DF
:102ED300F0F9FDFF7F3F3F7FFFFEF8F0C00000E009
:102EE300FFFFFFFF3F0100000000000000000000A3
:102EF300000000000080C0E0F0F8FCFE7F3F1F0FE1
:102F03000703010000000000013FFFFFFFFFE00394
:102F13007FFFFFFFF8800000000000000080C0E09A
:102F2300F0F8FCFE7F3F1F0F0703010000000000C5
:102F3300000000000000000080F8FFFFFF7F030097
:102F430000030F1F7FFFFEFCF0F8FCFEFF3F1F0F87
:102F53000703010000000000000000000000000063
:102F6300008080C0E0F0FCFEFF7F1F0F0300000025
:102F7300000000000000010307070F1F1F3F3E7EF4
:102F83007C7C7C7CFCF8F8F8F8787C7C7C7C3E3E8E
:102F93003F1F1F0F07070301000000000000001080
:102FA300010000007C92107C4444447C10927C001D
:102FB30000200400000000000000000000000000EA
:102FC300FCE28202020404080810A040A0100806D4
:102FD30006000000000000000000000000000000E8
:102FE300FFFFFFFEFCF8F8E4C28100000001020CC1
:102FF30030C00000000000000000000078FCFEFF6D
:10300300FFFFCF870707070707070707060604041D
:10301300040300000000183C3C3C3C3C3C3C3D3F6E
:103023003F3F3F3F3F3E3C3C3C3C3C3C3C3C3C18F0
:1030330000000012011001000000088304000000DA
:10304300010102000109092100010001222E0009EA
:10305300022200010100C0FA09040000010300007C
:1030630000092100010001222E0007058103080049
:103073006400002E06A0FF09A5A10109A609A51554
:1030830080257F75089540B10209A71580257F75B6
:10309300089508810209A91580257F750895409137
:1030A30002C0040309041A03570049004C004C00F2
:1030B3002000540052004E0049004300530000001A
:1030C3001803470050005300200041004C00450006
:1030D3005200540045005200FF30A5FF30A9FF30D5
:1030E300C30099A3ADB8C2CCD6E0EBF5009192939F
:1030F300949597999B9EDE0000000000000000005D
:10310300000000000000123B391242DAF111126094
:10311300BB1247FD126E23126FBCE4F522F523F5B3
:1031230021F5249087B9F0D20C90880D04F0124851
:1031330073020026310912518F124A5CEF640A7040
:103143006A124B05EF604824FA7060123EF5D12BEA
:103153009087A6E07002A3E07002B128900013E00C
:1031630054FDF0A20DB3920D90875BE07002A3E0D3
:10317300600312792C9087A6E07002A3E0600890A8
:10318300879BE0FF1256FF201921125205801C90E5
:103193000013E06402F01270B6126FDB51159087D2
:1031A3005BE07002A3E0600312792C1248733008CD
:1031B30028201A25201B22201C1F201D1C201E191D
:1031C300201F16C39087E7E0941E9087E6E09400E3
:1031D300400512464E8002C22030081F20201C20CA
:1031E3001A19201B16201C13201D10201E0D201F32
:1031F3000AF11190880BE0FF12529A1243151260E4
:10320300D4123BCB90841BE07002213C126DA002D0
:103213000033300802614790875DE004F0E0D39407
:10322300034002E4F0F1117A2F7BB4752C037D0483
:103233007F0571587871766E7871E6FFD394785074
:10324300157B017D0391687871E6FF7B3F7D0791D4
:103253006878710680E2787176037871E6FDD3941D
:103263000650157BFF7F6E91687871E6FD7BFF7FCB
:1032730078916878710680E290875DE07028752EFA
:10328300FF752F1275308312772F91607D037F288E
:10329300915E7D047F41915E7D057F32915E7D0667
:1032A3007F4DB10A40E490875DE06401702A752E7A
:1032B300FF752F1275308912772F91537D037F4845
:1032C300915E7D047F37915E7D057F30915E7D0643
:1032D3007F3F7158B11640E290875DE06402702829
:1032E300752EFF752F1275308F12772F91607D0326
:1032F3007F37915E7D047F4C915E7D057F41915EBA
:103303007D067F52B10A40E490875DE06403703428
:10331300752EFF752F1275309512772F91537D03FC
:103323007F2D915E7D047F4A915E7D057F43915E93
:103333007D067F3671587871E6FF7BFF7D049168C7
:10334300B10C40D8227E887F23125F377A2C7B838F
:10335300E4F52CFDFFF1F9F1EBE493787AF6F1EB68
:1033630074019308F6E47879F67979E7C3787B9664
:1033730040028127E47878F67878E6FFC3787A9676
:1033830040028122E52C701FE5282FFFE433FE184D
:10339300E6FD25291260601247F4C083C082F13C28
:1033A300E493FFEC4F8036E52C6401701612791D0F
:1033B3001260601247F4C083C082F13CE493FFECD7
:1033C3005F801AE52C6402701B12791D1260601273
:1033D30047F4C083C082F13CE493FFEC6FD082D00A
:1033E30083F08036787AE6FF18E6F98FF0A4F1EBE4
:1033F300A3A3258212781CF58318E6FFF15AE49300
:10340300FEEFFDE5282DFDE433FCE529291260607C
:103413002DF582E5833CF583EEF0787806617B78C1
:103423007906616CE528787A26FFE5290826FD9060
:103433008400EFF0A3EDF0EFD3947F400690840077
:10344300747FF0EDD3940740069084017407F02253
:103453007A2F7BA2752C037D027F5071587A2F7BC4
:10346300A2752C032275F080ED1260632FF15CE0EE
:103473004BF022F111787376037873E6FFC3947DE2
:1034830050157B017D0191687873E6FF7BE07D0633
:10349300916878730680E2787376027873E6FDC3E9
:1034A300940650177BFFE4FFF1E27F7FF1E27F7E1A
:1034B300F1E27F7D916878730680E07BFF7D01E414
:1034C300FF91687B3F7D06E4FFF1F27F0191687B0A
:1034D300607D067F01F1F27F0291687BE07D067FCC
:1034E3000291687BFC7D017F7FF1DB7F7F91687BAD
:1034F300FE7D017F7EF1DB7F7E91687BFF7D017F17
:103503007DF1DB7F7D816871587871E6FF7BFF7DFC
:103513000591687871E6FF7BFF7D069168787106F7
:10352300E6D3947822127841F11190882DE070024D
:10353300A3E0700C125A5990882DEEF0A3EFF022FD
:10354300201B4E7A887B237D167FBC7E02D11560BB
:1035530039E4D11E6034D21B123FD1752F00753070
:10356300061278DC124385714812512C90879BE038
:10357300C4540F75F00AA412718B95F040077F09AC
:103583007EB012513030B74C80FBE4D11E704580C1
:1035930040201C247A887B237D167F2C7E01D11545
:1035A300600FE4D11E600AD21C12512C12512C80E0
:1035B30023E4D11E701E8019201A197A887B23D127
:1035C3000F6009E4D11E6004D21A8008E4D11E7092
:1035D30003126FDB90882DE07002A3E060167A88F7
:1035E3007B23127900E4D11E6007E47FFFD11F70B3
:1035F30003126FDB301B14123FD1752F0075300699
:103603001278DC1243857148124E68227D5A7F0F6F
:103613007E00F16478711209C474FFFFFEFDFC782B
:10362300711209A7C30209671278419087B8E0FFB6
:10363300A3E004F0C39F4002E4F0126F97FF90876A
:10364300B9E0FE044F9000E0F0D2AFEE25E024A8ED
:10365300F582E43487F583E0FFA3E09087B6CFF0EB
:10366300A3EFF0F111125B81EF4E6025D21DC21E54
:10367300C21F7E877F927C887D2F126CE712512CAC
:10368300124E5912431590879BE0FF1270E720B743
:10369300FD9087A6E07002A3E06061301D5E201EEE
:1036A300297A877B927D167F2C7E01D1156014E4E5
:1036B300D11E600FD21E124E6890879BE0FF1271DD
:1036C3003C8023E4D11E701E8019201F197A877B4A
:1036D30092D10F6009E4D11E6004D21F8008E4D1A7
:1036E3001E70031270B67A877B92127900E4D11EA2
:1036F3006004D11C70031270B6124E5922F583E494
:10370300740193FA740293F9120A1E120026E478E4
:1037130076F6E47875F67875E6FFD3947F500E0855
:10372300E61260602FF15CE4F0180680E978760613
:10373300E6B408DEE4FDFF8132E0FC08E6FFED8F2E
:10374300F0A4852B82852A83A3A32582F582E583B2
:1037530035F0F5837878E62582F582E43583F583C1
:10376300228E27F1F9E4FFFEFDFC127944126975FC
:10377300127944126A15788EA607E6FFF460539017
:103783008837E0FBAD29125DAEEF6043127A14F582
:10379300831279E25009125E3BED24B4FB800A12D6
:1037A3007A14125E35AF05AB07788EE6FFAD2912AA
:1037B3005DAEEF6017AE27AF28E4FCFD788A12797F
:1037C300695005788A02098B74FF8007E48004E45A
:1037D3008001E4FFFEFDFC2291687BFF7D062291C0
:1037E300687873E6FD7BFF22852B82852A832291ED
:1037F300687B017D01228F288D298A2A8B2B22E465
:10380300900005F0900003F090000774FFF0E4903F
:103813000009F09000137407F09000157402F09003
:10382300001714F09000B07438F09000B47430F0C6
:103833009000C77401F0228C6F8D70E4FEF9BF0114
:10384300051241458011BF02051241358009BF03AE
:1038530004F1F78002517A74A0F011ABEBF053033B
:103863008011AB127A1EB503047E018005BC2002D1
:103873007901EE7003EC60E9E96401702811ABE0B3
:103883005480B503027E01BF01059025558013BF07
:103893000205904555800BBF030590655580039045
:1038A300855574F0F0AF0622857082856F83228F71
:1038B300658B688A69896ACEECCECFEDCF8E6D8F2A
:1038C3006EE56C156CAE6B7002156B4E602E127745
:1038D300127002056914F9120731FBAD6EAC6DAFBE
:1038E30065113A056EE56EAE6D7002056D14F582D5
:1038F3008E83E0FF908461E02FF080C52290849E48
:10390300E06002219190841CE024FD6002219190EB
:10391300849DE0FE7032EFD394014072EF24FFFDEB
:10392300E434FFFC908420E0FAA3E0FBC39DEA9C0F
:103933005008CCEACCCDEBCD8004EF24FFFD789E7C
:10394300EDF6EE0408F6801BEFFDC3908421E09DA5
:1039530031925005A3E0FF8000789EEFF690849D9E
:10396300E008F690841D124122789FE6249EF9E434
:103973003484FA7B0118E6756B00F56C11B2789EFE
:103983001277A4700990841CF0A3E0FF515D22908C
:103993008420E09400228F6590849CE06037E56585
:1039A3006002415C90845C7405F090841CE0908418
:1039B3005DF09000E0E090845EF09000E2E090849F
:1039C3005FF078DF7C847D017B017A84795C7E0003
:1039D3007F4002070B90841CE024FC705EE5657059
:1039E30020C3908421E0940731925005A3E0FF8027
:1039F300027F07789EEFF6756501E49084DFF0801F
:103A030016C3908421E0940831925005A3E0FF800F
:103A1300027F08789EEFF690841EE0FEA3E0FF7419
:103A2300DF2565127A96789EE6756B00F56C127643
:103A3300E11277A4702390841CF022E4789FF67837
:103A43009FE6FFC394085011E5652F24DFF582E458
:103A53003484F583E4F00680E622BF010512414574
:103A63008011BF02051241358009BF0304F1F780BD
:103A730002517A74F0F02290855574AAF0908AAAC4
:103A83007455F09085552271E3AB207D007C207F37
:103A93000151C8908803E0FB7D017C207F0151C860
:103AA300908812E0FB7D027C207F0151C890880E34
:103AB300E0FB7D037C207F0151C890880BE0FB7DF8
:103AC300047C207F018C298D2AE4FEF9BF010512B5
:103AD30041458011BF02051241358009BF0304F13E
:103AE300F78002517A74A0F0F1AFEBF0530380F149
:103AF300AF127A1EB503047E018005BC2002790152
:103B0300EE7003EC60E9E964017028F1AFE05480E2
:103B1300B503027E01BF01059025558013BF020541
:103B2300904555800BBF03059065558003908555DF
:103B330074F0F0AF0622902000E0F520300042E45C
:103B4300908803F09088127405F090880E7409F041
:103B5300E490880AF090880BF090880C740CF0C203
:103B630001C202C2001278F57D007C207F0171E35F
:103B73001279C8518A127A8651C4127A8E51C4D1ED
:103B8300CE902000E0F520A3E0908803F09020027F
:103B9300E0908812F0902003E090880EF0902004CB
:103BA300E090880BF0902005E090880AF0902006C2
:103BB300E090880CF0783B7C877D017B017A60790B
:103BC300007E007F0402070B3009147D007C207FF8
:103BD30001518A127A8651C4127A8E51C4C20922C3
:103BE3008C298D2AE4FEFDBF010A124145F1F090B4
:103BF3002AAA8020BF020A124135F1F0904AAA8016
:103C030013BF0309F1F7F1F0906AAA8007517AF123
:103C1300F0908AAA7455F0F1AF7430F0F1AF12410D
:103C23002BBB80047E018005BA20027D01EE700368
:103C3300EA60E9ED64017028AB04530380BB8002A2
:103C43007E01BF01059025558013BF0205904555A0
:103C5300800BBF0305906555800390855574F0F084
:103C6300AF0622E47872F6301102C11290841BE091
:103C73006002C11212371112678575321B75334802
:103C8300E4FB1258031265D0126F974401F0D2AFD0
:103C9300124873300119752EFF752F0F75304512B9
:103CA30079D812579C90873BD12B1257E280147519
:103CB3002EFF752F0F7530521279D890873BD12B79
:103CC300124FCA126CDE7B027D03E4FF12438B7832
:103CD30072E664017BFF7A1B79CA7028F1B6127908
:103CE3009112438B7BFF7A1B79CA12793BFFC37412
:103CF3003A9FFF752A017B3A7D03126000F1C412DB
:103D030078B58022F1B6127991F1E9F1C71278B54D
:103D13007BFF7A1B79CE12793B2443FB752A017D05
:103D2300037F43126000752EFF752F0F75305F758B
:103D330031FF75321C753305126CCA7B047D03E4B5
:103D4300FFF1E9F1C775320F75336A7B047D58E4DF
:103D5300FFF1E9752F0F75306C7531FF75321C75E6
:103D63003318907FFFE493FFC4540FF534EF540FDF
:103D7300F5357B057D03E4FFF1E9752F0F75307988
:103D83007531FF75321C7533217B067D03E4FFF12A
:103D9300E9752F0F75307E90800012099778111204
:103DA3000978EF541FFFE48F31120997781612092F
:103DB30078EF540FFFE48F32120997781A120978BB
:103DC300EF543FFFEF24D0F534E43407F5337B069B
:103DD3007D3FE4FF12438B301208E47872F6C2127F
:103DE300800930130678727601C213A210E433FF00
:103DF3007872E67E00B401027E01EE5F600C1278F9
:103E0300F51279C871E3D1CEC210124315816A222B
:103E13007872E6FE08E690D80475F00A1209DCEE23
:103E230075F00AA42583F583E0FCA3E0FDA3E0FE7F
:103E3300A3E0FF22301602C1CD123711D2169087AC
:103E4300D7127751127898D12B126AEA90882FD122
:103E53002B90874D1278EED12B9087511209D09079
:103E6300882FD12B9087431278EED12B908747125E
:103E730009D0127A559087D7D12B908722126C9E46
:103E8300F89087D7D12B1208C7908729124E3F90FD
:103E930087D7D12B126C85AF0590872AED124E4040
:103EA3009087D7D12B1208C7908728EBF09087F221
:103EB300E0908726124E40908722D12B126C85907A
:103EC3008727EDF0127ABD12371122E4FBFD7C60E7
:103ED3007F0351C8E4FB7D017C607F0351C8E4FB91
:103EE3007D027C607F0351C8E4FB7D037C607F031C
:103EF30041C8127841200802E1AE90882FD12B905F
:103F0300874D1278EED12B9087511209D09087E616
:103F1300E07002A3E060497E877F4D7C877D43127A
:103F23006CE7E47FE87E03FDFC7871127969500247
:103F3300800312784190873BD12B78711209A7EF48
:103F43002B1277E21278FA908737D12B7871120906
:103F5300A7EF2B1277E29087371209D0D20F803068
:103F6300C20FA20F300E01B350261279C871E3902D
:103F7300873BE0FB7D00D1EF90873CE0FB7D01D1E7
:103F8300EF90873DE0FB7D02D1EF90873EE0D1ECDF
:103F930090882FD12B9087431278EED12B908747AF
:103FA3001209D0300F03D20E22C20E22852A828537
:103FB30029832212000EEF75F006A4FFC3743B9F02
:103FC300FD752EFF752F0E7530BF7531FF22752ECF
:103FD300FF752F007530067531FF75321A7533CFB3
:103FE300E4FB7D1E7F0112438B752EFF227480F04C
:103FF30074AAF02290655574AAF0906AAA7455F0D9
:10400300906555228C658D66E4FEFDBF010A31453E
:10401300123FF0902AAA8024BF020A3135123FF0E2
:10402300904AAA8017BF030B123FF7123FF0906A22
:10403300AA8009123A7A123FF0908AAA7455F08541
:1040430066828565837430F0856682856583312B4E
:10405300BB80047E018005BA20027D01EE7003EA75
:1040630060E6ED64017028AB04530380BB80027EDD
:1040730001BF01059025558013BF0205904555806A
:104083000BBF0305906555800390855574F0F0AF21
:10409300062290849EE06073B4050890849C7401AA
:1040A300F08022781C7C847D017B017A84799E7E5A
:1040B300007F4012070B7E007F407D007B017A84E6
:1040C300795C120A2490849EE024FD603224FD6012
:1040D3002514601914601B14600924087028E4F582
:1040E300AE801790841B7401F0E4A3F022310FE437
:1040F300800831188004310F311890841CF022900D
:10410300849F31221107E4FF1239992290849FE0A2
:104113009000E0F0229084A0E09000E2F0E422E03E
:10412300FFA3E0FCA3E0FD22E0FCFB5420FA5303D1
:10413300802290455574AAF0904AAA7455F0904590
:10414300552290255574AAF0902AAA7455F090250B
:104153005522C0E0C0F0C083C082C0D075D018E53E
:10416300E830E111E5EA30E609E5ED543060035348
:10417300EABF53E8FDE5E830E45843EA3853EADFA1
:104183009084DEE0FFC394405043C374409FFFC359
:104193009408500280027F08789BEFF69084DEE05B
:1041A30024DF127A96EFFD7C0012750F53E8EF7847
:1041B3009BE6FF9084DEE02FF0C394404005127726
:1041C3001B800F9084DEE0FF1239998005518753DD
:1041D300E8EFE5E830E37DE5ED30E6181276A07808
:1041E3009DEFF653E8F7E6606B127660EF706512A9
:1041F300732B8060E5ED540F605490849DE0C3946D
:1042030040504BE5ED540F789BF6087600789BE61B
:10421300FF08E6FEC39F501490849DE02E249EF574
:1042230082E43484F583E5EFF00680E163ED8053A7
:10423300E8F7123900789BE6FF90849DE02FF0C3E6
:1042430094404010119553EA9043EA20800663EDB1
:104253008053E8F7E5E830E20612754353E8FBE5DF
:10426300E830E00353E8FEE5E830E70353E87FE591
:10427300E830E50553E8DF51B0D0D0D082D083D009
:10428300F0D0E032127420EF7022908817E0B4056A
:1042930015A3E0FF4480F5EEEF90881F60057403DB
:1042A300F080037402F090881774FFF022127650A6
:1042B30075E10275EA3875EA1875EC0C75EB28752B
:1042C300E6BA75E6BE75EB2275E9BF75EE80F5E8D3
:1042D30075B70143A7012290881212676F90880E69
:1042E30012724B51ED12731E80C37F0112607180F5
:1042F30021752F1A7530377531FF75321C753336BA
:10430300908839E0F534A3E0F5357B057D05E4FFBE
:10431300718BE4FF12608DE47875F67875E6FFC360
:104323009408504E126099E47876F67876E6FFC3E7
:1043330094805039EFC394405009C2C5D2C4EF7082
:1043430011800BD2C5C2C47876E6B44005E4FF12EF
:1043530060A8D297C2C2D2C67876E6FF18E612608A
:10436300602F12375CE0126092080680BE787506F3
:1043730080A922752F1A7530297531FF75321A7588
:10438300339F7B027D1E7F018F2B8D2C8B2DE49021
:104393008767F0A3F0A3F0A3F07875762908760C6D
:1043A300F540754100754231852E43852F44853094
:1043B300458540468541478542487B017A84790299
:1043C3001219BD127832FF7002A117E52B705DEF51
:1043D30024E0908769F0A37406F0E4A3F0F1C340EE
:1043E30002A104908768E0FDE52C2DFDE433FCEE8B
:1043F3007E002DFFEE3C1279BD4002A10490876B35
:10440300E0F9908769E075F006A42455F582E5F09C
:10441300341CF583E5822912375CE493FD75F08043
:10442300E52D126063F1F4EDF1D780B1E52B640162
:10443300704212783224E0127A5E241FF582E5F08E
:10444300342412775CE490876BF0F1C3501E12772B
:10445300ED501912780BF583C083C08290876BE00F
:10446300FFD082D083126039F1CE80DEF1EC64029A
:1044730070D3A104E52B64026002A104127832FF19
:1044830064206047EF24D0127A5E240CF582E5F0B5
:10449300342912775CE490876BF0F1C3501E1277D6
:1044A300ED501912780BF583C083C08290876BE0BF
:1044B300FFD082D083126039F1CE80DEF1EC640349
:1044C30070D390876AE02402F0803690876A740E76
:1044D300127778E490876BF0F1C35020EE252CFF20
:1044E300E433FE908768E07C002FFFEC3E1279BD39
:1044F300500A12605AF1F4E4F1D780DCF1ECB40312
:10450300D290876AE0FF908768E02FF0908767E09A
:1045130004F061C6E52B7008908768F1DF04801210
:10452300E52B908768B40106F1DF24028004F1DFF4
:104533002403FD0234328F277A2E7B77752C037D7B
:10454300037F67123358E527C4540F30010E7E00F2
:10455300540FFF124F4C8E318F32800312795F75E7
:104563002EFF752F1A7530257B037D6FE4FF718B4A
:10457300E527540F14B407004002C1439045861247
:1045830071317302459B0245B00245D10245E702F2
:1045930045FD02461E024630D1447531FF75321A7D
:1045A300753385E4FB71877A2B7B7FC140D14475DA
:1045B30031FF75321A75338C123FE3D1477531FFE2
:1045C30075321A75338571857A2C7B01806FD144DE
:1045D3007531FF75321A753395123FE371767A2C74
:1045E3007B838059D1447531FF75321A7533A91213
:1045F3003FE371767A2C7B838043D1447531FF7519
:10460300321A7533B2123FE3D1477531FF75321A4F
:104613007533BD71857A2C7B838022752EFF752FB0
:104623001A75302C1272E47A2C7B838010752EFF5E
:10463300752F1A7530301272E47A2C7B8312335340
:1046430022752EFF752F1A7530292290883BE0FFC3
:1046530020E70520E602E1A612371190883BE0FD32
:10466300C4540F90883FF0ED30E71220E40720E5B3
:10467300045430600890883F7408F0C22090883B4F
:10468300E0540F90883DF0700204F07A2C7B837520
:104693002C03E4FD7F02123358F1A77532197533E9
:1046A30082E4FB7D26123FE7F1AA75321975338840
:1046B300E4FB7D647F01718B300116752EFF752F2E
:1046C3001975308B1278C4FD124F578E318F32809B
:1046D3000C752EFF752F197530921257D77185906F
:1046E300883FE024FB7002E17214605F14603414AD
:1046F3006002E1A1F1A7753219753399F1B4123F44
:10470300E9F1AA75321975339F7B047D487F0271E5
:104713008B2020067F22F1BB80777F1B7EB0125156
:1047230030806EF1A77532197533A3F1B4123FE9E6
:104733001278237D6E7F02718B2020067F21F1BBCF
:1047430080077F1B7EB01251308046F1A775321966
:104753007533AFF1B4123FE9127823F1E620200656
:104763007F20F1BB80077F1B7EB01251308022F186
:10477300A77532197533B6F1B4123FE9127823F1F4
:10478300E62020067F1FF1BB80077F1B7EB01251FE
:104793003071157FC07EC67D2D7C000250EA123732
:1047A30011C22022752EFF752F1975307F7531FFC9
:1047B300227B04E4FD7F02227EB0125130D22022FC
:1047C30090876AE0FFA3E0FEC39F222DF582E58375
:1047D3003CF583EEF090876BE004F022E0252CFF9C
:1047E300E52D227D647F02618B90876CE004F0E00D
:1047F300222FF582E5833EF58322C2AFD2A8C2B849
:10480300C289D2885389F0438902758CADE4F58A55
:10481300D2B9D28CD2A9F5C8D2BD75CD6375CB639D
:1048230075CCC075CAC0D2ADD2CAC299C28E4387F5
:104833008053890F438920758DECD28E90851FF0AC
:10484300908520F0759850C299C298D2ACD2BC75AD
:10485300913075950343972075948875B10875B2A7
:104863000775B30875B40775A131D2AF43A71022FA
:10487300300C3C90880DE025E025E04422F597E5D7
:104883009730E0FB90880DE0FF14600804700B90F4
:1048930088058003908802E596F0EFC394015008E1
:1048A30090880DE004F08005E490880DF0C20C229E
:1048B300C0E0C0F0C083C082C0D075D000C000C0CB
:1048C30001C002C003C004C005C006C007C2A87867
:1048D300AA760020B20878AAE6D3942340F578AAF2
:1048E300E6D3942350213127EF601C3127EF601763
:1048F3003127EF60123127EF600D3127EF60083168
:104903006A90883E7405F0D2A8D007D006D005D0AF
:1049130004D003D002D001D000D0D0D082D083D035
:10492300F0D0E032E478AAF630B20878AAE6D3945D
:104933002340F578AAE6FFC3940E4028EFD39414DE
:104943005022E4F620B20878AAE6D3942340F578FF
:10495300AAE6FFC394004009EFD3940650037F01F6
:10496300227F00227F0022E4FF7E01FDE478AAF685
:1049730030B21278AAE6FCD394235009EC94234076
:10498300EF7EFF80EBEF25E0FF78AAE6FCC3940BF4
:10499300400BECD3941150054307018013ECC394EF
:1049A30004400BECD3940A50055307FE80027EFFAC
:1049B300E478AAF620B20878AAE6D3942340F578DF
:1049C300AAE6D3942340027EFF0DED6408709DEEAA
:1049D300F4601090883BEFF0E0C4540F7002C220E3
:1049E3007F01227FFF22C0D075D008C28C78AA062F
:1049F300D28CD0D032C0E0C083C082C0D075D0107A
:104A030030981EC29890851FE02401FFE433FE9086
:104A13008520E06F7001EE600890851F512DE599A8
:104A2300F0D0D0D082D083D0E032E0FF04F0742104
:104A33002FF582E43485F58322908520E0FF90856D
:104A43001FE0C39F70037FFF22C2AF908520512DCB
:104A5300E07872F6D2AFE6FF22513C7871EFF6F4BC
:104A6300600FE6FF600B908621E0FE04F05196EFA5
:104A7300F07871E6FFF46006EF6003B40ADB90861A
:104A830021E0600C2421F582E43486F583E0FF22E3
:104A93007FFF2274222EF582E43486F58322F1E827
:104AA30090876504F0908621E024FBFF908765E002
:104AB300FEC39F5015A3E0FF5196E0FEEF6E908773
:104AC30066F0908765E004F080DB908766E0FF1274
:104AD30072F6908621E0241FF582E43486F583E0A4
:104AE300B5071C908766E0FF127308908621E024C7
:104AF3001EF582E43486F583E0B507037F01227F48
:104B03000022787176FF752AFF752B00752C697565
:104B13002D00752E067B017A8679221218D4EF7048
:104B23001A51A1EF60157148EF600C787176062079
:104B33001609123E378004E47871F6E4908621F07A
:104B43007871E6FF22E4FFFEFDFC7872F13C787693
:104B5300F13C787A1209C47E867F22F196B19FF1E7
:104B630096B1BE1203CB9087651209D09087651268
:104B73003E2B9087D71209D0F1A49087D7123E2BF2
:104B830090875E126C9EF89087D7123E2B1208C74F
:104B9300908763EFF0E070037418F0D1419087D7EA
:104BA300123E2B126C85AF05908764EDD140908740
:104BB300D7123E2B1208C7908762EBF078A6E6FE69
:104BC30008E6FFD122908769B1B0D137F163F1884C
:104BD300C000787212098BD000F169787612098BC4
:104BE300E412038D126CF7120169F1E012027212E2
:104BF30013FD7BCE7A6379DE7842120169D15112BB
:104C03000272D13712016990872D1209D0F17B12FC
:104C1300083CC004C005C006C007787212098BD0D7
:104C230003D002D001D000F1B3F171C004C005C0BC
:104C330006C007D148120169D003D002D001D000C9
:104C430012007890876AD11190876EB1B0D137F195
:104C530063F188C000787212098BD000F169F17B8F
:104C630012083CC004C005C006C007787212098B45
:104C7300D003D002D001D000F1B3F171C004C0055C
:104C8300C006C007D148120169D003D002D001D0B9
:104C93000012007890876FD111908773B1B012031F
:104CA300CBAD07AC06E41203927B187A0979EDF1D8
:104CB30061908774EEF0A3EFF04E600BE02405F0F3
:104CC300908774E03400F0F1A4B19F78A6A606089B
:104CD300A607908774E07002A3E0700A9087E8E06B
:104CE300908776F0802778A4E6FE08E6FF78A7E6AB
:104CF30024FFFD18E634FFFCB1D8126D007C017D62
:104D03006812079BECC313ED13908776F078A6B176
:104D1300B21203CB9087771209D090876EE0B45319
:104D23000F90876A123E2B12037C90876A1209D078
:104D3300908773E0B4570F90876F123E2B12037C5A
:104D430090876F1209D0C208908769E06441704967
:104D530078D77C877D017B017A877965FE7F161280
:104D6300070B9087DC123E2B90882F1209D0908777
:104D7300E1123E2B9088331209D09087E8E09088A7
:104D830037F0E4A3F0D2089087D7127751127898BE
:104D9300123E2B126AEA7F01227F00220FEFAC063C
:104DA30070010E14F5828C83E0B42CF022F008E637
:104DB300FE08E6FF78A4A60608A607B19F78A6EE2C
:104DC300F6FC08EFF6FD78A4E6FE08E6FFED24FF07
:104DD300FDEC34FFFC8E278F288C298D2A787B7C71
:104DE300877D017BFF7A3079FA7E007F0F12070BF4
:104DF300C3E52A9528FFE5299527FEAA27A9287B3D
:104E030001787B7C87F1D87A87797B02193712097D
:104E1300D078A6E6FE08E6FF78A4A60608A607B1A2
:104E23009F78A6A60608A60778A4E6FE08E6F582FC
:104E33008E83E022E4FBFA797A784422EFF0E47B74
:104E430064FAF9F822787612098BE412038DE4FBF5
:104E5300FA796178452290879BE0FF1245397E8776
:104E63007F92125F37787112098B126CEE752EFFE9
:104E7300752F1275305EF1F07B057D4B7F02123F7B
:104E8300E9752F12753063852A34852933852832D5
:104E93008527317B067D767F0112438BE47F64F1A6
:104EA30024500B752EFF752F12753065806AF13310
:104EB300D141D31209675012E47FC8F124500B7516
:104EC3002EFF752F1275306B804EF133E47BC8FAD9
:104ED300F9F8D31209675014E47F2C7E01F12550B1
:104EE3000B752EFF752F12753071802CF133E47B17
:104EF3002C7A01F9F8D31209675014E47F907E01EC
:104F0300F125500B752EFF752F12753077800975BB
:104F13002EFF752F1275307D7B05E4FD7F02024362
:104F23008BFEFDFCAB2AAA29A928A827C30209677F
:104F3300AF2AAE29AD28AC27221209C4E4FFFEFD37
:104F4300FC2290880CE0FF7E007C007D0A1207891A
:104F5300AC06AD07E41203927BDB7AF9791E783F46
:104F63001201690203CB1208C778760209C4E4FB75
:104F7300FA797078420201697FA07E867D017C0008
:104F830078760209A778721209C47BA07A86790120
:104F930078002278A6EEF608EFF678A4A60608F6BF
:104FA3002278A6E6FE08E6FF78A4A60608A607224E
:104FB300C3EF9BFFEE9AFEED99FDEC98FC787A1215
:104FC30009C4787A12098BE412038DE4FBFA797A27
:104FD30078440202727D0112070B7B0122E4FBFA83
:104FE3007934784322E4908765F0A3F0228F348EDE
:104FF300338D328C3122C0E0C0F0C083C082C0D078
:1050030075D008C2CF908804E4F0E5C0F4540325BA
:10501300E025E0FFE590F454034FF0E0FF908811A2
:10502300E0FE6F6021EF600E90880FE4F090872020
:1050330004F0A374F4F090880FE0C39496502FEE1D
:10504300602C42228028EE60259087207401F0A313
:1050530074F4F090880FE0FFC394965002800CEF35
:10506300B4960BD214EE422290880FE004F090889D
:1050730004E0908811F0908720E07002A3E0600EB6
:10508300908721E024FFF0908720E034FFF09088A0
:1050930001E004F0E0C394324004E4F0D20C9088C1
:1050A30006123E2BEC4D4E4F601C908806A3A3A323
:1050B300E024FFFFEE34FFFEED34FFFDEC34FFFC94
:1050C3009088061209D090883EE0600214F0D0D098
:1050D300D082D083D0F0D0E0327F1B7EB031307FDE
:1050E300C07EC67D2D7C008F2B8E2A8D298C28E4D3
:1050F3007F207E4EFDFCAB2BAA2AA929A828C31228
:1051030009674024E47B207A4EF9F8AF2BAE2AAD31
:1051130029AC281208C79088061209D09088061275
:105123003E2BEC4D4E4F70F4227F1D7EB0300214A7
:10513300D374189F74B09E500BEF941EEE94B0502E
:10514300037F00227876A60608A60720B7FDD2B50E
:10515300C2B4C2B60000E47875F6127A6EEE30E798
:1051630004D2B48002C2B4C2B5EF25E07977F7EE7A
:105173003319F70000D2B50000787506E6B410DAEB
:10518300C2B40000D2B630B7FD7F0122752EFF7581
:105193002F137530937B017D13E4FF123FE9752FC5
:1051A3001375309C7B027D117F02123FE9752F132B
:1051B3007530A47531FF75321B7533E37B057D1C98
:1051C3001243112002147F1B7EB031307F0C7EB05E
:1051D30031307FC07EC67D2D80067F807E847D1E1C
:1051E3007C0011EA90883EE060127F1FF1A47F20CB
:1051F300F1A47F21F1A47F227EB03130126D190218
:1052030037111278AA9087E6E0300111FCA3E0FD84
:10521300124F57127A7E124F45F1FB800A1279EC36
:1052230090880CE01279A7127A4C605812799C404E
:105233004F201852D3ED944AEC9401503F1237118A
:10524300518D12797C123FE7752F1375308D7531AF
:10525300FF12777FE69400400CF1D075307F127710
:10526300D27D5C80051277C77D607F0112438B126C
:10527300431511DC11DC11DCD218800AC218800638
:10528300C2188002C2187F0122FD752EFF752F12EE
:105293007530237531FF228F271267F9C39087E793
:1052A300E0944A9087E6E09401400F90872BE0FF5B
:1052B300A3E09087E6CFF0A3EFF0E5276402600256
:1052C30061D3518D75321A75335CFBFDFF12438B2D
:1052D300300119127A0A1278C4FD124F578E318F9A
:1052E3003212784B752F1275309F800E127A0AF1A5
:1052F300D712784B752F127530A3127A67518D75BB
:10530300321B7533D2D1F79087E8E0F4700261BEA7
:10531300E0FF740BD39F5011E0C39421500B752E03
:10532300FF752F127530A761CA12695F5011E0C370
:105333009438500B752EFF752F127530AE61CA125B
:1053430069555011E0C3944E500B752EFF752F1203
:105353007530B5807212694B5011E0C39465500BE0
:10536300752EFF752F127530BC805C126941501188
:10537300E0C3947B500B752EFF752F127530C380DD
:10538300461269375011E0C39492500B752EFF7586
:105393002F127530CA803012692D5011E0C394A8C2
:1053A300500B752EFF752F127530D1801A752EFF95
:1053B300752F127530D89087E8800C752EFF752FE6
:1053C300127530DF9087E81269697D0A7F02C1CCCC
:1053D300E52764016002A1FB518D75321B7533A56E
:1053E3007B01FDFF12438B300115752EFF752F12C4
:1053F3007530E6F19C908737123E2BF1E2801275EF
:105403002EFF752F127530EF908737123E2B124FF8
:10541300CA124FF01279CF518D75321C75334F7B01
:1054230002E4FDFF123FE9752F127530F8908726CD
:10543300F1DA7B027D1CE4FF123FE9752F1375300F
:10544300037531FF7532137533109087F2E0F5342D
:10545300A3E0F5357B027D3AE4FF123FE9519075F5
:10546300321B7533DA7B03D1F9300115752EFF75C5
:105473002F13753012F19C90873B123E2BF1E28083
:1054830012752EFF752F1375301B90873B123E2B21
:10549300124FCA124FF07B037D26E4FF12438B5158
:1054A3008DD1F1300116752EFF752F13753024122F
:1054B30078C4FD124F578E318F32800B752EFF75D6
:1054C3002F1375302CF1D77B04127AC490872912DD
:1054D30069FE12785DF89087281277DC90873F1277
:1054E30009D09087631269FE12785DF89087621283
:1054F30077DC90871C1209D090873FF1C490871CFA
:10550300127751C39BFFEE9AFEED99FDEC98FC9048
:1055130087571209D0518D75321C7533497B05D1DC
:10552300F9908737123E2BEC4D4E4F6042300119F4
:10553300127A001279B2F1C412083C908757F1C471
:105543001208C7F19CF1E2801C1279F61279B2F1CC
:10555300C412083C908757F1C41208C7F19C120883
:10556300C7E412038D124FF07B057D2CE4801230CB
:105573000105127A0080031279F6E4F5317B057D8B
:105583002CFF12438B518DF1F47B06D1F9127A76FD
:105593007C007D0A30010E124F501278E6752F13EE
:1055A300753024800C1207891278E6752F13753035
:1055B3002C7B06127AC4518D75321B7533DE7B0743
:1055C300D1F9126F84752F137530489087F0E0F589
:1055D300319087EFE0F5327B07E4FF123FE9752F47
:1055E300137530527531FF75321375335D126CCA02
:1055F3007B077D4BE4FFC1CC518D75321B7533A501
:10560300E4FBFDFF12438B300115752EFF752F133D
:10561300753061F19C908737123E2BF1E280127551
:105623002EFF752F13753069908737123E2B124F5B
:10563300CA124FF01279CF518DF1F47B02D1F99058
:10564300880CE0FF602730010E124F4A1278E6758E
:105653002F13753071801090880CE012795F752ECE
:10566300FF752F137530787B037D3280137BFF7AB0
:105673001A797912793BFFC3745A9F518C127A2895
:10568300E4FF12438B518DD1F1300121F1D07530FC
:105693007F1278C4FD124F578E318F327B057D2DDB
:1056A3007F02123FE9752F1275309F8016F1D07576
:1056B300307FF1D77B057D2D7F02123FE9752F12D5
:1056C3007530A37B067D5E7F0112438B9087F2E0EA
:1056D300FF908732E06F6003127ABD127A5590878C
:1056E300E6E0FFA3E090872BCFF0A3EFF022753223
:1056F3001A75335C7B04E4FDFF02438B8F2712781A
:10570300AA9087E6E030011BFCA3E0FD124F57127D
:105713007A7EE527C4540F7E00540FFF124F4CF1DD
:10572300FB800B1279ECE527C4540F1279A7127A88
:105733004C606112799C405820195BD3ED942CEC9A
:1057430094015048123711752EFF752F137530834E
:105753007531FF12797C123FE7519012777FE694FF
:1057630000400CF1D075307F1277D27D5C8005123A
:1057730077C77D607F0112438B1243157F1A11DEB9
:105783007F1A11DE7F1A11DED219800AC218800631
:10579300C2198002C2197F0122E47BE87A03F9F877
:1057A300227EB031307F807E847D1E7C0001EA1230
:1057B30009DCEE75F00AA42583F583120997908816
:1057C3002FE0F8A3E0F9A3E0FAA3E0FB22752EFF94
:1057D300752F13229087E6E0F531A3E0F53222120C
:1057E30008C7E412038D7BDB7AF9791E783F020147
:1057F3006975321B75331E227871A60608A6072227
:105803007F0112438B752A017B7FE4FDFF7874A629
:10581300077874E6D39B503EE52A7018F1F11260C5
:10582300632F12375CE0440212788412375CE04441
:1058330040F0801DE52A640170177874F1F112605D
:10584300632F12375CE0F412788412375CE0647FD4
:10585300F078740680BB22E47872F608F630110201
:10586300413190841BE060024131127854752F0E50
:105873007530EA1278DCE4FB7F0112438B908839A0
:10588300E07002A3E0701A752A017B7FFDFF1110FF
:10589300123FC475321B7533F97B047D19E4FF2174
:1058A300E9752EFF752F0E7530FA7873E62401F52E
:1058B3003218E436F531E4FB7D6611035132123EB2
:1058C3001C513C1203117872600250075134123E8E
:1058D3001C80085134123E1C12037C124E51127963
:1058E30052EFF05132123E1C513C1203119087D5F6
:1058F3006002500E5144C004126A0E5132123E1C13
:1059030080185144C004C005C006C0075132123E7E
:105913001C12037CD003D002D001D0001278715145
:1059230032123E1C513C1203117F53600250027F1E
:105933004E8F31752EFF752F0F753000127744F59A
:1059430037126CE07B02127A9E123E13513C120313
:1059530011787260025005123E158006123E151230
:10596300037C124E51127952EFF0123E13513C1246
:1059730003119087D56002500C5144C004126A0E83
:10598300123E1380165144C004C005C006C007125E
:105993003E1312037CD003D002D001D000127871E1
:1059A300123E13513C1203117F57600250027F4590
:1059B3008F31752EFF752F0F753019127744F53718
:1059C300126CE07B04127A9E7872F1F87173F5839E
:1059D300E075F002127962752EFF752F0F75303264
:1059E3007B067D077F0112438B12647E301317D32E
:1059F3007873E6940018E69400400708E6161870DA
:105A03000116C2130160201202016090883AE0245B
:105A1300FFFF908839E034FFFEC37873E69F18E6F2
:105A23009E50070806E618700106C212016022782C
:105A330072E6FE08E690D80022E4FBFAF9F874F067
:105A430022E0FEA3E0FFE4FCFD7B107A0EF9F812DE
:105A5300083CE402038D908839E07002A3E07002F1
:105A63006165E47875F608F67875F107126FB29EF2
:105A73005002616590D80075F00AEF123E1FF11EC7
:105A830078C11200781257C174F0120311500261E9
:105A93005B78755134123E1CF11E78411200781266
:105AA30057C174F012031160044002615B787512F0
:105AB3003E157B927AB1790978C2F1EA1257C47420
:105AC300F01203115002615B7875123E157B927AD6
:105AD300B179097842F1EA1257C474F012031160E4
:105AE300025075787551347173AF82FE7C887D2FB7
:105AF300126A157877A607E6FFF4605CF10E60582A
:105B03007875E6FE08E6FF90D8087173F583E0C365
:105B130074809480501390D80875F00AEF7176D191
:105B230035AF05ED24B4FB800C7875F1F87173D1B2
:105B330035AF05AB077877E6FFF113601B78755136
:105B4300347173FAA9827B0178237C88F12EE49067
:105B5300882CF078760270AD787606E61870010628
:105B6300416B126FDBE4FEFF22E6FE08E6907FFE48
:105B730075F00A1209DCEE75F00AA4258322127A65
:105B8300B5F1DB127AA5E4081278ADF1D408120955
:105B9300C4F1D47882124F3C78861209C4126FFD87
:105BA300787AEEF608EFF6D39414EE9400500512CB
:105BB3007AB5800A787BE624EC79771270A5F1DB5D
:105BC300FF24ECFDEE34FFFC787AE6FA08E6FBC32B
:105BD3009DEA9C40097878A60608A607800AEB246C
:105BE300147879F6E43A18F6F1DBFF4E7002A1AAB5
:105BF300EB4A7002A1AA7878EAF6FC08EBF678760D
:105C0300A60408F64A6006E61618700116EF6B70D4
:105C130002EE6A6008787906E618700106D3787791
:105C2300E6940118E694004023787A716CF11978B0
:105C3300C1120078787612790E717A127987600C26
:105C4300400A7877E6161870011680D17878F10744
:105C53009087B7E09F9087B6E09E402008716CF173
:105C6300197841120078787812790E717A1279874F
:105C7300500A787906E61870010680D0127A6E7899
:105C83007AA60608A607787AF107787996EE189629
:105C93005075907FFE75F00AEF7176F1259087A419
:105CA300E0B4EE03127A437E877F9C7C887D2F12BB
:105CB3006975787E1209C47E877F9C126D0CF4602F
:105CC3003CF10E60389087A41279E25008D13BED85
:105CD30024B4FB80099087A4D137AF05AB0778754F
:105CE300E6FFF1136017127AAD123624400F127AD1
:105CF300AD1209C4787AE6FE08E6127AA5787B0627
:105D0300E6187001068189787DE618467002A1AA1B
:105D1300E47F207E03FDFC78821279694002A1AA08
:105D2300787C716CF1259087A4E0B4EE03127A437A
:105D33007A877B9C7D0F7FBC7E0212376478861244
:105D430009C4F1D47886123624605CE4FFFEFDFCBE
:105D5300788612362460509087B9E0FFE4FCFDFE9C
:105D63007BCC7A0CF9F812083CEF787D26FFEE180D
:105D730036FE787AF608EFF69087A6E06E7003A3F6
:105D8300E06F6023787AE6FF08E69087A6CFF0A35A
:105D9300EFF07A87799C7B0178927C87F12E90874C
:105DA300A6E0FEA3E0FF22E4FEFF228F2CAA051249
:105DB3007970C3648094805008D13BED24B4FF8094
:105DC30007127970D13BAF05788FA607EA252CFF20
:105DD300E433FEC3648094805008D13BED24B4FFC8
:105DE300800BE52C2AFFE433FED13BAF057890EF1F
:105DF300F618E6FEB507037F01227890E6FFEED39F
:105E03009F401B18E6D39B5006EBC394B44009E4B0
:105E1300D39B5007EB9F50037F01227F0022788F93
:105E2300E6D39B500A08E6FFEB9F50037F01227FD6
:105E33000022F583E0FF7E007C007DB40207F09032
:105E43008839E0FAA3E0FBC39433EA94034002C128
:105E5300DD90882F123E2B90D800127A3A717AF592
:105E6300831278EE123E2B90D804127A3A717AF5A7
:105E7300831209D0908837E0C374809480500AD18C
:105E830037AF05ED24B4FF8007908837D137AF05CE
:105E9300126FA990D80875F00A1209DCEC717AF533
:105EA30083EFF090D809127A31717AF583E4F09098
:105EB300883AE004F07006908839E004F09088395D
:105EC300126F6CF1E37531FF75321A7533DD7B02A6
:105ED300123FE71242F47F0A8018126F73F1E375E1
:105EE30031FF75321A7533E67B02123FE71242F433
:105EF3007F187EB01251307F407E4B7D4C7C000278
:105F030050EA7876E6FE08E6FFD322908837E0FB76
:105F13007D16B1AEEF22F5831209977B1C7A347993
:105F2300CF22FAA9827BFF789C7C877D017E007F4C
:105F33000A02070B126D0C908837E0D39F4012EFD3
:105F430024B4FFE433FEE0FDC3EF9D7877F6EE80E3
:105F53000E908837E0FF7875E6C39F7877F6E49470
:105F63000018F6F105740B9FE49E500FC3EF9421C4
:105F7300EE940050067A2E7B2D804CF10574219F00
:105F8300E49E500FC3EF9438EE940050067A2D7BB5
:105F9300E38034F105747B9FE49E500FC3EF94922A
:105FA300EE940050067A2D7B99801CF10574929F24
:105FB300E49E500FC3EF94A8EE940050067A2D7B15
:105FC3004F80047A2D7B05752C03E4FD7F67023334
:105FD3005874FFFFFEFDFC229087B6E0FEA3E0228B
:105FE300752F1A7530342212007890883322E6FF19
:105FF30075F080ED22E6FE08E690D808227873A6B5
:10600300077873E6FFD39B502CE52A701075F08058
:10601300ED11632F12375CE04402F08013E52AB4DC
:10602300010E7873125FF111632F12375CE0F4F005
:1060330078730680CC222582F582E43583F5837458
:106043000193FEEFFDE52C2DFDE433FC908768E022
:106053007A002DFDEA3CFC90876CE0252D75F080DD
:10606300A42400F582E5F03480F583E58222D297FB
:1060730000118400EF443E900005F000C29722D245
:1060830097C2C2C2C6D2C5D2C4221182EF44C09005
:106093000005F0C29722AE071182EE44B811929028
:1060A3008401EEF022AE07D297C2C2C2C6EE4440CC
:1060B3001192908400EEF022E47871F67871E6FF95
:1060C300C394FA500B74222F124A99E4F00680EC21
:1060D30022300813A210B014500D9087E8E0F4604A
:1060E30004514371B1C210A211B01450067175313D
:1060F3000B800FA2137212500CC212C2131237116B
:10610300D1D0123711020026301102412A90841B8C
:10611300E06002412A908720E07002A3E070024110
:106123002AE49087D4F0123FC475321A7533FCFB0E
:10613300FD7F0112438BE47871F67871E6FFD39407
:106143007F500C7B407D0112346878710680EBE44C
:106153007871F6513B5038EF7192FDEF7183FC512A
:106163002B75F012A424C4F9740FF17712438B78C2
:1061730071E6512C716DB50611E6FE7192FFEE7159
:1061830083FD752A017B7F12581078710680C41233
:10619300431530133B51439087D1E0D39400402CF7
:1061A300E014F0E47871F6513B500E512B716DB54C
:1061B3000602716678710680EE715F600FE4787194
:1061C300F6513B5007512B14F00680F5C213803C67
:1061D30030123951439087D1E0C39405502CE00429
:1061E300F0E47871F6513B500E512B716DB50602F8
:1061F300716678710680EE715F600FE47871F65115
:106203003B5007512B04F00680F5C21220100221E7
:106213000B71759087D1E075F003A42463F582E4D4
:106223003410123700210B22EF75F003A424C7F5B5
:1062330082E43487F583E0227871E6FFC394032276
:106243007F197EB0025130301102614690841BE009
:10625300600261469087D4F0F18575321B75333740
:10626300E4FB125803E47872F67157503FEF75F070
:1062730003A424BFF582E43487F583E0FD71A1FC18
:10628300714775F011A42430F97410F17712438B20
:106293007872E6FF7148FE9087D0E0FDEEB5050702
:1062A30071A1FBB160918378720680BD917E30133A
:1062B3003B51439087D0E0D39400402CE014F0E4AA
:1062C3007872F67157500E7147717BB5060271668D
:1062D30078720680EE715F600FE47872F671575042
:1062E30007714714F00680F5C213803C3012395110
:1062F300439087D0E0C39402502CE004F0E478721A
:10630300F67157500E7147717BB50602716678724C
:106313000680EE715F600FE47872F6715750077173
:106323004704F00680F5C212201002414A717590AD
:1063330087D0E075F003A42475F582E43410123796
:1063430000414A22EF75F003A424BEF582E43487AA
:10635300F583E0227872E6FFC39403229087D4E0AA
:106363006401229087D47401F022FF9087D1E0FE6C
:10637300EF22120026023711FF9087D0E0FEEF22B2
:1063830075F003A424C9F582E43487F583E022750C
:10639300F003A424C8F582E43487F583E022EF7583
:1063A300F003A424C0F582E43487F583E0229088C7
:1063B30039E07002A3E07002816F124FE8126FA000
:1063C300908765E0FCA3E0FDC39FEC9E4002816FD4
:1063D30090D800127A31123E237B1C7A34794F789D
:1063E300C01200781257C174F0120311406E9176F7
:1063F30090D800123E1C7B1C7A34794F78401200EF
:10640300781257C174F01203116002504F917690C5
:10641300D804123E1C7B927AB1798978C0125FEA64
:106423001257C474F01203114032917690D80412BB
:106433003E1C7B927AB179897840125FEA1257C485
:1064430074F012031160025013908766E02401FF79
:10645300908765E03400FE126EC48013908766E077
:1064630004F07006908765E004F061C0125E42E4B8
:10647300FEFF22908765E0FEA3E022B1D002431520
:106483007D057F0102438BE47872F690880BE0F67A
:10649300301102A15890841BE06002A1589084003F
:1064A300E0123FC375321B75330CE4FB1258033003
:1064B300131290880BE0D394004005E014F0D20946
:1064C300C213801330121090880BE0C3940250055E
:1064D300E004F0D209C212752EFFB1C675321B75E6
:1064E30033AC7B027D05123FE7B1C675321B7533B2
:1064F300B57B047D05123FE7B1C675321B7533C109
:106503007B06918390880BE07006B1607B02801854
:1065130090880BE0B40106B1607B04800B90880B7C
:10652300E0B40206B1607B069183301024C2109060
:10653300880BE07872F6123711126F73123FC7752A
:10654300321C75332A127A671243151250E212373E
:1065530011917E81937872E690880BF022752EFF5D
:10656300752F0E7530C622908400E0123FC375323A
:106573001B75335AE4FB125803B1D02011449084A5
:106583001BE0703E301206D1BFC2128007301304E5
:10659300D1BFC213752EFF752F0F75308A7B037D14
:1065A30005123FE7752F0F7530987B059183200106
:1065B30006B1607B038004B1607B059183124315B0
:1065C30080B922752F0E7530C27531FF22E47874BD
:1065D300F67874E6FFD3947F500C7B807D071234EA
:1065E3006878740680EB787476017874E6FDD3944A
:1065F3000750177BFFE4FF1234687874E6FD7BFFD6
:106603007F7F12346878740680E022F1851257F494
:10661300E4FB125803B1D0301102C1BE90841BE0D9
:106623006002C1BE30121290880CE0C39421500561
:10663300E004F0D209C212801330131090880CE0EA
:10664300D394004005E014F0D209C213752EFF75F0
:106653002F0E7530CC7B03918390880CE0604A2029
:106663000113752EFF752F0E7530DCD1C7127A76A4
:10667300126EBD800E752EFF752F0E7530E4D1C7D7
:10668300124F451278E6752F0E7530E07B031243E7
:1066930087752EFF752F0E7530E87B037D0A123F39
:1066A300E7B1637B037D6E8008123FC4127A287DB5
:1066B300087F0112438B124315C11A22A201B39220
:1066C30001D209227B037D467F0102438B90840024
:1066D300E012528C75321A75333DE4FB125803B144
:1066E300D0301002E16B90841BE0707C908720E037
:1066F3007002A3E06072301214908812E0C3940A0F
:106703005004E004F16C12512CC2128015301312A4
:10671300908812E0D394004004E014F16C12512CE1
:10672300C213752EFF752F127530269088121272C0
:106733003F123FE7752F1275302B12725A7871F69C
:106743007871E6FFC3940A501A908812127234507B
:10675300067A297BBD80047A297BA712722C787173
:106763000680DD124315C1E422F0D209E09030E443
:1067730093F5A22235F0752EFFF52F8930AB047FF8
:106783000122908400E0FD752EFF752F0E7530C831
:106793007531FF22F18575321B75337EE4FB125888
:1067A30003B1D020114790841BE07041301206F1F1
:1067B300F1C2128007301304F1F1C2133002111237
:1067C30078CC75337A7534FF75351A753679800F41
:1067D3001278CC75337A7534FF75351A75366D7B3F
:1067E300037D0A7F0112438B12431580B622A20256
:1067F300B39202D209227A297BF5752C03E4FD7F3B
:10680300621233589087E8E0F470022113E0FF74BA
:106813000BD39F501DE0C3942150177A2B7B193162
:1068230025311B70022113752EFF752F1275302D24
:106833002107315F5022E0C39438501C7A2A7B91A0
:10684300752C037D017F6B311B70022113752EFFA5
:10685300752F1275303321073155501DE0C3944E07
:1068630050177A2A7BF73125311B70022113752EBD
:10687300FF752F127530392107314B501BE0C3943C
:106883006550157A2A7BB3311470022113752EFFDC
:10689300752F1275303F806C3141501BE0C3947BE0
:1068A30050157A2B7B5D3125311B6064752EFF7586
:1068B3002F12753046804D3137501BE0C3949250F0
:1068C300157A2A7BD53125311B6045752EFF752F2F
:1068D3001275304C802E312D5019E0C394A85013FB
:1068E3007A2B7B3B31146028752EFF752F12753080
:1068F3005280117A2A7B6F31146015752EFF752F24
:10690300127530589087E831697D61E4FF12438B3B
:1069130022752C037D017F6A12335890880BE06443
:106923000222752C037D017F69229087E8E0FF74C2
:1069330092D39F229087E8E0FF747BD39F229087B6
:10694300E8E0FF7465D39F229087E8E0FF744ED39D
:106953009F229087E8E0FF7438D39F229087E8E076
:10696300FF7421D39F22E025E0F532E433F5317B38
:10697300052291A8E4FFFEFDFC788F124F3C78932B
:10698300124F3C78971209C4852F82852E831257A4
:10699300C4852D82852C83123E2B1200747B9A7A38
:1069A3001979F77841120169789391BB1257C49111
:1069B300B1123E2912007490872D1257C412016937
:1069C30078971209C4789712098B510C120169C088
:1069D30004C005C006C007789312098B510C12013D
:1069E30069D003D002D001D000120078121735B15C
:1069F30000788F1209C4788F02098BE0FF7E007C38
:106A03000E7D10120789E4FCFDA804A905AA06ABB4
:106A1300072291A8852F82852E831257C48F828ED9
:106A230083123E2B120074788F91BB1257C491B11D
:106A3300123E2912007478931209C4789312098BB9
:106A430091DE788F12098B121861124FE0120169DF
:106A530091F7120272510CE4FFFE7DE17C431200B8
:106A6300741203CB7897EEF608EFF651C7500D1862
:106A730051DEED2468FFEC3401FE800B789751DE84
:106A8300ECC313FEED13FF7897A60608A607E4FFF1
:106A9300FEFDFC789351CE700DFFFEFDFC788F5107
:106AA300CE70037FFF2251D651C77D0050027D0176
:106AB300ED6009125E3BED24B4FF800751D6125EF0
:106AC3003BAF0522C3EE64809480221209A774F0C1
:106AD3000203117897E6FE08E6FF22E6FE08E6FFCA
:106AE3007C017D680207F091EE124E411208C7EB5C
:106AF30024D0FEEA34079087EDF0A3CE124E401265
:106B03004F3391859087EFEDF091A1F8124F331237
:106B130008C79087F0EFF091A1F8917C1208C79015
:106B230087F2124E3F917C91859087F3ED124E4090
:106B3300917C1208C79087F4EBF0916454037018AA
:106B4300FC7D6412079BED4C70089164918FED4CB2
:106B530070069087F6741DF09087F2E0F9FF339585
:106B6300E0FEAD2FED3395E0FCEF2DFFEE3CFEC3D1
:106B7300EF9418EE648094804026916DFD9087F029
:106B8300E004F0D39D40119087EFE004F0A3E0FD13
:106B9300916DFCED8CF091969087F2E0252F802784
:106BA30051C750299087F0E014F09400501190875A
:106BB300EFE014F0A3E0FF916DFEEF8EF09196905D
:106BC30087F2E0252F241875F01884800AE52F2911
:106BD30075F018849087F2E5F0F09087EDE0FAA362
:106BE300E0FB7C017D6DFFAE02120789AC06AD07A9
:106BF300EBAE027802CEC313CE13D8F92DFBEC3ED5
:106C030091639188C3EB9FFBEA9E9163918FEF2B76
:106C1300FFEE3ACF2494CF34FEFE7C007D071207AB
:106C23009B9087F1EDF0787E76019087EFE0FF7817
:106C33007EE6FEC39F501574F42E9173FF9087F187
:106C4300E02F75F00784E5F0F00680DE9087F1E031
:106C530014FF9087F0E02F75F00784A3E5F0F0228E
:106C6300FA9087EDE0FEA3E0FF229087EFE024F4A3
:106C7300F582E43487F583E022AF2EAE2DAD2CAC44
:106C83002B221208C77C007D6402079B7C017D9048
:106C930002079B849087F0E5F0F0221209D0E47B91
:106CA300107A27F9228E2C8F2D8C2E8D2F22E52DF5
:106CB3002404F582E4352C221209C4E52F2404F5BB
:106CC30082E4352EF58322908802E0FCE4120397D8
:106CD3007B857AEB79C7783D1201698F378E368DC4
:106CE300358C3422317578710209C48F2A8E298D2F
:106CF300288C27227BDC7A0F7949784022E4FBFA3F
:106D0300F9783F1200780203CB7C887D2F511578E8
:106D130075A607E6FF22E4F52790298DB1947A2919
:106D23007B8DB184B18C40F1124315B1A0E4F527FA
:106D330090299AB1947A297B9AB184E47FD07E0713
:106D4300FDFC1250EA124315B18C40E4752EFF7519
:106D53002F137530AB7531FF75321B7533EF7534F7
:106D6300FF75351B7536CA7B057D1712431120024B
:106D73000C7F007EB012513030B70580FB1257A84C
:106D830022752C037D060233580527E527C3940992
:106D930022E493FFE5278FF0A4240FFF22E47F1062
:106DA3007E27FDFC0250EA8F27E47872F6F19745BF
:106DB30027F0D2AF7A8079067BFFC001E52775F013
:106DC30002A424A6F9748735F0A801FC7D01D00143
:106DD300D11CD10EE0FEA3E0FFF47002EEF46004D8
:106DE300EF4E700BD10EE4F0A3F07872F6800478C6
:106DF300727601D10EE0FEA3E0FF9087B7E02FF09B
:106E03009087B6E03EF07872E6FF22E52725E0247E
:106E1300A6F582E43487F583227E007F0202070B06
:106E230078397C887D017B017A407900D11CF1A0FF
:106E33004E6025C3EF9433EE94035011D1BD780017
:106E43007CD87D017B017A40790202070BE49088AC
:106E530039F0A3F0FFFED15C228E278F287C407D82
:106E6300007F02123BE37C407D00908839D1B67CE1
:106E7300407D0190883AD1B6E47873F608F6AE27E0
:106E8300AF28D1BDC37874E69F18E69E50247E4098
:106E9300E6FA08E6FB2402FD74403AFC74002BF585
:106EA3008274D83AF583D1B6787406E61870010671
:106EB30080CC22E0FB7F02023AC87C007D0A0207F5
:106EC30089F1A9D39400EC9400407D90882DE0B51E
:106ED3000607A3E0B50702F18FED6F7002EC6E6059
:106EE3003CEF64014E60361257FB7871125F07F175
:106EF300B29E4029D1BD74002FF974D83EFA7B01AC
:106F0300C00174F62FF974D73EA801FC7D01D001AE
:106F1300125F30787206E61870010680CD90883AC9
:106F2300E024FFF0908839E034FFF0F16C125FE366
:106F33007531FF75321A7533EC7B02123FE712424B
:106F4300F47F0B125EF5801EF173125FE37531FF60
:106F530075321A7533F67B02123FE71242F47F183B
:106F6300125EF57F00227F0122E0FEA3E0FFD15CE9
:106F73001234767A297BD3752C037D027F0A123370
:106F830058908400E02405FD752EFF22E490882D9F
:106F9300F0A3F022C2AF9000E0E054F822908839C9
:106FA300E0FEA3E0FF22908839E0FCA3E0FD2290FD
:106FB300883AE09F908839E022787176017871E60B
:106FC300FFD394075011B1AAEF60077871E6908759
:106FD300B8F078710680E622F18FC21BC21CC21A78
:106FE300FFFEFDFC9088231270DE9088271209D0E3
:106FF30090882B74FFF0E4A3F022E4788AF608F675
:10700300125FDBFF24FF788DF6EE34FF18F6EF4EA8
:10701300700201A1788CE6FE08E6FF788AE6FC0898
:10702300E6FDD39FEC9E5072ED2FFFEC3EC313FEA3
:10703300EF13FF788EEEF608EFF608A60608F66D56
:107043007002EC6E6054788EE6FE08E6FF788D667B
:10705300700318E66E604390800875F00AEF1257CC
:10706300B274F0120311500B788FE624FF798D115F
:10707300A580A1788EE6FE08E690800875F00A12D6
:1070830057B274F01203116011400F788FE6240198
:10709300798BF718E43619F701177891800CE4FE21
:1070A300FF22F718E634FF19F722E62401FF18E45C
:1070B30036FE22E49087A6F0A3F0C21DC21EC21FB3
:1070C300C219FFFEFDFC90879211DE90879612098C
:1070D300D090879A74FFF0E4A3F0221209D0E4FF62
:1070E300FEFDFC22317E94004043ED604014B40762
:1070F30000503A9070FC3131730271110271150224
:10710300711902712902711D0271210271257F011A
:1071130080167F0280127F04800E7F03800A7F0621
:1071230080067F0780027F057EB01251302275F002
:1071330003A4C58325F0C58322317E9400403BED33
:1071430014B40700503490714F31317302716402EB
:10715300716602716A02717602716E027172027156
:107163007280007F0F800E7F10800A7F1080067F61
:107173000D80027F107EB012513022EF540FFDEFCD
:10718300C4540F75F00AA4FEFFC39087E7E09F90F5
:1071930087E6E022301102412B90841BE06002411C
:1071A3002B12678575321B753325E4FB12580330A8
:1071B300121490880EE0C3940A5007E004F0D20939
:1071C300514BC212802030131D90880EE0D39400DF
:1071D3004012E014F0D209E09030EF93FFF5AA7467
:1071E300FF9FF5ABC213752EFF752F0F75303E90C1
:1071F300880E513F123FE7752F0F753043515A7870
:1072030072F67872E6FFC3940A501890880E5134D0
:1072130050067A297BBD80047A297BA7512C78728A
:107223000680DF124315219722752C037D05023357
:1072330058E0FEEFC39E908400E0FF22E075F00A61
:10724300A4F5317B037D4B22E09030EF93FFF5AA49
:10725300C374FF9FF5AB227B037D647F0112438BD5
:107263007D057F0A123432E42212678575321B755D
:10727300336CE4FB1258031265D020116390841B16
:10728300E0705D301214908803E0C36480948C50E6
:1072930005E004F0D209C21280153013129088035E
:1072A300E0D3648094744005E014F0D209C21390D3
:1072B3008803E0FFC364809480400D752EFF752F13
:1072C3000F7530A88F31800F752EFF752F0F753016
:1072D300B3908803E0F5317B0351EF124315809A95
:1072E300227531FF75321A7533C7E4FB7D197F01AF
:1072F30002438B53070FEFD39409EF50042430FF5D
:10730300222437FF225307F0EFC4540FFFD394090D
:10731300EF50042430FF222437FF22D2B5D2B6C265
:10732300B4D2C32275EAB022D150A3E05460701ADC
:10733300A3E024FB600E14600D24FD600B24087091
:107343000902002E80DE800681EF43EA4022908806
:1073530019E024FE602214602D24E2605614606359
:107363002421707891CC7430F0A37436F090881493
:10737300E4F0A37412F0806891CC7430F0A37452DB
:10738300F09030548039908818E075F003A424DB22
:10739300F582E5F03430F583E493FB740193FA74DA
:1073A3000293F9908820EBF0A3EAF0A3E9F0120727
:1073B30031801E91CC7430F0A37449F0903048E4CE
:1073C30093800E91CC7430F0A37477F0903076E410
:1073D30093FF908814E4F0A3EFF0800443EA402283
:1073E30090881DE0FE90881CE0FDEDFF789EEEF690
:1073F300FE08EFF6908814E0FCA3E0FDC391E57F5F
:107403000050027F01908813EFF0789E125F07ED22
:1074130091E54006A3EEF0A3EFF053EA7F908820B6
:10742300A3E0FAA3E0F9EA49700281C6908814E068
:10743300FEA3E0FF4E700691DCF5EA807A78A2EEB7
:10744300F608EFF6D391D440061876000876089133
:10745300DCFF78A3E64FF5EAE478A0F608F6C379F3
:10746300A1E778A39618E66480F819E7648098503A
:107473001F908820E0FBA3E475F001120826A9F011
:10748300FA120731F5E778A106E61870010680CEF7
:1074930078A2E6FE08E6FFC3908815E09FFD90887A
:1074A30014E09EFCF0A3EDF04C7015908813E0609F
:1074B30006C3EF91D45009908820E4F0A3F0A3F021
:1074C3007F012275EA907F002290882074FFF0A349
:1074D300229408EE6480948022E5EA648054804418
:1074E30030229FEE6480F8EC64809822908818E044
:1074F300D3940090881F40077404F0B1098003748B
:1075030003F075EAB022B14353EADF228B658A6642
:107513008967D3ED9408EC6480948040047C007DFB
:107523000891DC4DF5EAED1DAE0470011C4E600FB1
:10753300D1477002056614F9120731F5E780E72297
:10754300789E760008760778A9E690878AF0C37458
:107553002496FFE41896FED374079FEE6480F874B4
:1075630080984007789EEEF608EFF6789EE6FE08D0
:10757300E6FF78A8E6FC08E62422F974863CFA7B49
:1075830001788B7C87124FD87A87798A756A007560
:107593006B087F017E00B1BC789EE6FE08E678A802
:1075A3000826FFF618EE36FEF6C3EF9424EE648049
:1075B30094804004E4F608F6228E658F668B678A12
:1075C30068896943EB28E566640145657006D13B2C
:1075D3004002800CE56664024565700AD13B4006B3
:1075E300756A00756B08E478A0F608F6C378A1E61F
:1075F300956BE56A6480F5F018E6648095F0501C9D
:10760300AB670569E569AA687002056814F9120792
:1076130031F5E60806E61870010680D0E5EB6480D4
:1076230054804420FFE566640245657E0070027E57
:1076330040EF4E456BF5EB22D3E56B9408E56A64A6
:1076430080948022AB650567E567AA66229088204F
:10765300E4F0A3F0A3F0908814F0A3F0229088162E
:10766300E0FEB4210DA3E0B40908E490849DF07F0B
:107673000122EE64A17023908817E0B4011C53EA41
:107683007F7B017A8479DF7D087C00B10F9084DEF3
:107693007408F0FF1239997F01227F00227565017A
:1076A300756688756716E5ED540F6408600643EA4E
:1076B300407F0022E4789EF608F6D1477002056603
:1076C30014F9E5EF120777789F06E618700106783C
:1076D3009FE66408184670E243ED807F01228B68C1
:1076E3008A69896AE56C156CAC6B7002156B4C602A
:1076F3001D0FEFCCEECC70010E14F5828C83E0FDF0
:10770300F1127002056914F9ED12077780D622ABE6
:1077130068056AE56AAA692290849CE06002E4F045
:1077230090841CE06005E4FF123999227531FF75DE
:10773300321A75334EFBFD7F0112438B7871766EDF
:10774300229087D5E0F532A3E0F5339087BAE0FCC9
:10775300A3E0FDA3E0FEA3E022F583740193FA7492
:107763000293AE02FF7875EEF608EFF6F5828E838C
:10777300E49390876AF0E490876CF02275321A756F
:10778300335C7B047D037F0112438B7A2E7B8075F0
:107793002C037D017F50123358C37872E69464182A
:1077A30022E6FF7E0090841FE02FF090841EE03ECF
:1077B300F0C3908421E09FFF908420E09EFEF0A31D
:1077C300EFF04E22752EFF752F137530897871E611
:1077D300F53108E6F5327B0322E0FFE4FEEB2FFFF1
:1077E300EE3AFEED39FDEC38FC22EEFDE52C2DFDE5
:1077F300E433FC908768E07A002DFDEA3CFCD3ED8E
:10780300947FEC648094802290876CE08FF0A4FFD7
:107813007875E6FC08E68C832FF582E58335F02244
:10782300752F197530AB90883DE0F5317B042290BC
:107833008767E02402F582E43484F583E022E4FFE1
:10784300FEFDFC78710209C47B017D0A7F021243AD
:107853008B908400E0FD752EFF22A3E075F03CA41D
:10786300FFEB2FFBEA35F0FAED39F9EC3822120081
:1078730074E4FBFA797078421202729087BA0209B3
:10788300D0F075F080EDA42480F582E5F03480F526
:1078930083E5822F22F52E8E2D8D2C8C2B90880341
:1078A300E0F52F9087E922E47871F608F608F608E8
:1078B300F62275321B7533CE7B037D44E4FF02430E
:1078C3008B9087E6E0FCA3E022752EFF752F0F75E2
:1078D30030BE7531FF75321B227531FF75321A7553
:1078E30033D6228E318F32752EFF221209D0908823
:1078F3003322E4FFFEFDFC90873B0209D07D167F17
:10790300207E0312376478710209C4E6FA08E69010
:107913007FFE75F00A1209DCEA227878E62528FF53
:10792300E433FE08E6FD25292290875CE024FFF07E
:1079330090875BE034FFF02212000EEF75F006A48F
:1079430022788A1209C47C887D2FAF2BAE2A22129B
:1079530002721203CB9087D5EEF0A32275F00AA42E
:1079630085F031F532221209A7D3020967EAFFC372
:10797300E52C9FFFE49400FE2275321A7533657B74
:10798300027D0322F5831209B474F00203117532E8
:107993001B7533CA7B03E4FF2208E6FC08E6FDC33C
:1079A3009FEC9E2275F00AA47871A6F008F622E4F3
:1079B3007F107E0EFDFC90873722FED3EF947FEE7F
:1079C30064809480227D007C607F03227B017D2C78
:1079D300E4FF02438B7531FF75321C75334322E09C
:1079E300FF7E00C37480948022FEA3E07873A60612
:1079F30008F622752EFF752F1375303E22752EFF64
:107A0300752F1375303422752EFF752F1275309B29
:107A130022E52B2408F582E4352A22E0FD5420FCDC
:107A2300ED5480FA2275321A7533797B032275F08F
:107A33000AED1209DCEC2275F00AEB1209DCEA22EA
:107A4300908837E09087A4F0227871E6FE08E6FF7D
:107A53004E229087F2E0908732F022908769F0758A
:107A6300F003A4227B027F0102438B7876E6FE08B3
:107A7300E6FF2290880CE0FF7E00227873A60608BA
:107A8300A6072290880AE0FB7D052290880CE0FB84
:107A93007D0622F9E43484FA7B01227D077F01020B
:107AA300438BFF08A60608A60722787E12098B7867
:107AB300822278767600087601227F1E7EB00251FC
:087AC300307D32E4FF02438B29
:027FFE0015204C
:00000001FF
